
06_uart_modular.elf:     file format elf32-littlearm

Sections:
Idx Name          Size      VMA       LMA       File off  Algn
  0 .isr_vector   00000198  08000000  08000000  00010000  2**0
                  CONTENTS, ALLOC, LOAD, READONLY, DATA
  1 .text         000012e0  080001a0  080001a0  000101a0  2**4
                  CONTENTS, ALLOC, LOAD, READONLY, CODE
  2 .rodata       000000a4  08001480  08001480  00011480  2**2
                  CONTENTS, ALLOC, LOAD, READONLY, DATA
  3 .ARM.extab    00000000  08001524  08001524  00020064  2**0
                  CONTENTS
  4 .ARM          00000000  08001524  08001524  00020064  2**0
                  CONTENTS
  5 .preinit_array 00000000  08001524  08001524  00020064  2**0
                  CONTENTS, ALLOC, LOAD, DATA
  6 .init_array   00000004  08001524  08001524  00011524  2**2
                  CONTENTS, ALLOC, LOAD, DATA
  7 .fini_array   00000004  08001528  08001528  00011528  2**2
                  CONTENTS, ALLOC, LOAD, DATA
  8 .data         00000064  20000000  0800152c  00020000  2**2
                  CONTENTS, ALLOC, LOAD, DATA
  9 .bss          00000038  20000064  08001590  00020064  2**2
                  ALLOC
 10 ._user_heap_stack 00000604  2000009c  08001590  0002009c  2**0
                  ALLOC
 11 .ARM.attributes 00000030  00000000  00000000  00020064  2**0
                  CONTENTS, READONLY
 12 .debug_info   000028fe  00000000  00000000  00020094  2**0
                  CONTENTS, READONLY, DEBUGGING, OCTETS
 13 .debug_abbrev 00000769  00000000  00000000  00022992  2**0
                  CONTENTS, READONLY, DEBUGGING, OCTETS
 14 .debug_aranges 00000150  00000000  00000000  00023100  2**3
                  CONTENTS, READONLY, DEBUGGING, OCTETS
 15 .debug_ranges 00000108  00000000  00000000  00023250  2**3
                  CONTENTS, READONLY, DEBUGGING, OCTETS
 16 .debug_macro  0000fa27  00000000  00000000  00023358  2**0
                  CONTENTS, READONLY, DEBUGGING, OCTETS
 17 .debug_line   0000198b  00000000  00000000  00032d7f  2**0
                  CONTENTS, READONLY, DEBUGGING, OCTETS
 18 .debug_str    00055289  00000000  00000000  0003470a  2**0
                  CONTENTS, READONLY, DEBUGGING, OCTETS
 19 .comment      00000053  00000000  00000000  00089993  2**0
                  CONTENTS, READONLY
 20 .debug_frame  00000bdc  00000000  00000000  000899e8  2**2
                  CONTENTS, READONLY, DEBUGGING, OCTETS

Disassembly of section .text:

080001a0 <__do_global_dtors_aux>:
 80001a0:	b510      	push	{r4, lr}
 80001a2:	4c05      	ldr	r4, [pc, #20]	; (80001b8 <__do_global_dtors_aux+0x18>)
 80001a4:	7823      	ldrb	r3, [r4, #0]
 80001a6:	b933      	cbnz	r3, 80001b6 <__do_global_dtors_aux+0x16>
 80001a8:	4b04      	ldr	r3, [pc, #16]	; (80001bc <__do_global_dtors_aux+0x1c>)
 80001aa:	b113      	cbz	r3, 80001b2 <__do_global_dtors_aux+0x12>
 80001ac:	4804      	ldr	r0, [pc, #16]	; (80001c0 <__do_global_dtors_aux+0x20>)
 80001ae:	f3af 8000 	nop.w
 80001b2:	2301      	movs	r3, #1
 80001b4:	7023      	strb	r3, [r4, #0]
 80001b6:	bd10      	pop	{r4, pc}
 80001b8:	20000064 	.word	0x20000064
 80001bc:	00000000 	.word	0x00000000
 80001c0:	08001468 	.word	0x08001468

080001c4 <frame_dummy>:
 80001c4:	b508      	push	{r3, lr}
 80001c6:	4b03      	ldr	r3, [pc, #12]	; (80001d4 <frame_dummy+0x10>)
 80001c8:	b11b      	cbz	r3, 80001d2 <frame_dummy+0xe>
 80001ca:	4903      	ldr	r1, [pc, #12]	; (80001d8 <frame_dummy+0x14>)
 80001cc:	4803      	ldr	r0, [pc, #12]	; (80001dc <frame_dummy+0x18>)
 80001ce:	f3af 8000 	nop.w
 80001d2:	bd08      	pop	{r3, pc}
 80001d4:	00000000 	.word	0x00000000
 80001d8:	20000068 	.word	0x20000068
 80001dc:	08001468 	.word	0x08001468

080001e0 <memchr>:
 80001e0:	f001 01ff 	and.w	r1, r1, #255	; 0xff
 80001e4:	2a10      	cmp	r2, #16
 80001e6:	db2b      	blt.n	8000240 <memchr+0x60>
 80001e8:	f010 0f07 	tst.w	r0, #7
 80001ec:	d008      	beq.n	8000200 <memchr+0x20>
 80001ee:	f810 3b01 	ldrb.w	r3, [r0], #1
 80001f2:	3a01      	subs	r2, #1
 80001f4:	428b      	cmp	r3, r1
 80001f6:	d02d      	beq.n	8000254 <memchr+0x74>
 80001f8:	f010 0f07 	tst.w	r0, #7
 80001fc:	b342      	cbz	r2, 8000250 <memchr+0x70>
 80001fe:	d1f6      	bne.n	80001ee <memchr+0xe>
 8000200:	b4f0      	push	{r4, r5, r6, r7}
 8000202:	ea41 2101 	orr.w	r1, r1, r1, lsl #8
 8000206:	ea41 4101 	orr.w	r1, r1, r1, lsl #16
 800020a:	f022 0407 	bic.w	r4, r2, #7
 800020e:	f07f 0700 	mvns.w	r7, #0
 8000212:	2300      	movs	r3, #0
 8000214:	e8f0 5602 	ldrd	r5, r6, [r0], #8
 8000218:	3c08      	subs	r4, #8
 800021a:	ea85 0501 	eor.w	r5, r5, r1
 800021e:	ea86 0601 	eor.w	r6, r6, r1
 8000222:	fa85 f547 	uadd8	r5, r5, r7
 8000226:	faa3 f587 	sel	r5, r3, r7
 800022a:	fa86 f647 	uadd8	r6, r6, r7
 800022e:	faa5 f687 	sel	r6, r5, r7
 8000232:	b98e      	cbnz	r6, 8000258 <memchr+0x78>
 8000234:	d1ee      	bne.n	8000214 <memchr+0x34>
 8000236:	bcf0      	pop	{r4, r5, r6, r7}
 8000238:	f001 01ff 	and.w	r1, r1, #255	; 0xff
 800023c:	f002 0207 	and.w	r2, r2, #7
 8000240:	b132      	cbz	r2, 8000250 <memchr+0x70>
 8000242:	f810 3b01 	ldrb.w	r3, [r0], #1
 8000246:	3a01      	subs	r2, #1
 8000248:	ea83 0301 	eor.w	r3, r3, r1
 800024c:	b113      	cbz	r3, 8000254 <memchr+0x74>
 800024e:	d1f8      	bne.n	8000242 <memchr+0x62>
 8000250:	2000      	movs	r0, #0
 8000252:	4770      	bx	lr
 8000254:	3801      	subs	r0, #1
 8000256:	4770      	bx	lr
 8000258:	2d00      	cmp	r5, #0
 800025a:	bf06      	itte	eq
 800025c:	4635      	moveq	r5, r6
 800025e:	3803      	subeq	r0, #3
 8000260:	3807      	subne	r0, #7
 8000262:	f015 0f01 	tst.w	r5, #1
 8000266:	d107      	bne.n	8000278 <memchr+0x98>
 8000268:	3001      	adds	r0, #1
 800026a:	f415 7f80 	tst.w	r5, #256	; 0x100
 800026e:	bf02      	ittt	eq
 8000270:	3001      	addeq	r0, #1
 8000272:	f415 3fc0 	tsteq.w	r5, #98304	; 0x18000
 8000276:	3001      	addeq	r0, #1
 8000278:	bcf0      	pop	{r4, r5, r6, r7}
 800027a:	3801      	subs	r0, #1
 800027c:	4770      	bx	lr
 800027e:	bf00      	nop

08000280 <main>:
#include "uart.h"




int main(void){
 8000280:	b580      	push	{r7, lr}
 8000282:	af00      	add	r7, sp, #0
	uart2_tx_init();
 8000284:	f000 f8b6 	bl	80003f4 <uart2_tx_init>
	while (1){
		printf("hello.. \n\r");
 8000288:	4801      	ldr	r0, [pc, #4]	; (8000290 <main+0x10>)
 800028a:	f000 f997 	bl	80005bc <iprintf>
 800028e:	e7fb      	b.n	8000288 <main+0x8>
 8000290:	08001480 	.word	0x08001480

08000294 <_read>:
	_kill(status, -1);
	while (1) {}		/* Make sure we hang here */
}

__attribute__((weak)) int _read(int file, char *ptr, int len)
{
 8000294:	b580      	push	{r7, lr}
 8000296:	b086      	sub	sp, #24
 8000298:	af00      	add	r7, sp, #0
 800029a:	60f8      	str	r0, [r7, #12]
 800029c:	60b9      	str	r1, [r7, #8]
 800029e:	607a      	str	r2, [r7, #4]
	int DataIdx;

	for (DataIdx = 0; DataIdx < len; DataIdx++)
 80002a0:	2300      	movs	r3, #0
 80002a2:	617b      	str	r3, [r7, #20]
 80002a4:	e00a      	b.n	80002bc <_read+0x28>
	{
		*ptr++ = __io_getchar();
 80002a6:	f3af 8000 	nop.w
 80002aa:	4601      	mov	r1, r0
 80002ac:	68bb      	ldr	r3, [r7, #8]
 80002ae:	1c5a      	adds	r2, r3, #1
 80002b0:	60ba      	str	r2, [r7, #8]
 80002b2:	b2ca      	uxtb	r2, r1
 80002b4:	701a      	strb	r2, [r3, #0]
	for (DataIdx = 0; DataIdx < len; DataIdx++)
 80002b6:	697b      	ldr	r3, [r7, #20]
 80002b8:	3301      	adds	r3, #1
 80002ba:	617b      	str	r3, [r7, #20]
 80002bc:	697a      	ldr	r2, [r7, #20]
 80002be:	687b      	ldr	r3, [r7, #4]
 80002c0:	429a      	cmp	r2, r3
 80002c2:	dbf0      	blt.n	80002a6 <_read+0x12>
	}

return len;
 80002c4:	687b      	ldr	r3, [r7, #4]
}
 80002c6:	4618      	mov	r0, r3
 80002c8:	3718      	adds	r7, #24
 80002ca:	46bd      	mov	sp, r7
 80002cc:	bd80      	pop	{r7, pc}

080002ce <_write>:

__attribute__((weak)) int _write(int file, char *ptr, int len)
{
 80002ce:	b580      	push	{r7, lr}
 80002d0:	b086      	sub	sp, #24
 80002d2:	af00      	add	r7, sp, #0
 80002d4:	60f8      	str	r0, [r7, #12]
 80002d6:	60b9      	str	r1, [r7, #8]
 80002d8:	607a      	str	r2, [r7, #4]
	int DataIdx;

	for (DataIdx = 0; DataIdx < len; DataIdx++)
 80002da:	2300      	movs	r3, #0
 80002dc:	617b      	str	r3, [r7, #20]
 80002de:	e009      	b.n	80002f4 <_write+0x26>
	{
		__io_putchar(*ptr++);
 80002e0:	68bb      	ldr	r3, [r7, #8]
 80002e2:	1c5a      	adds	r2, r3, #1
 80002e4:	60ba      	str	r2, [r7, #8]
 80002e6:	781b      	ldrb	r3, [r3, #0]
 80002e8:	4618      	mov	r0, r3
 80002ea:	f000 f877 	bl	80003dc <__io_putchar>
	for (DataIdx = 0; DataIdx < len; DataIdx++)
 80002ee:	697b      	ldr	r3, [r7, #20]
 80002f0:	3301      	adds	r3, #1
 80002f2:	617b      	str	r3, [r7, #20]
 80002f4:	697a      	ldr	r2, [r7, #20]
 80002f6:	687b      	ldr	r3, [r7, #4]
 80002f8:	429a      	cmp	r2, r3
 80002fa:	dbf1      	blt.n	80002e0 <_write+0x12>
	}
	return len;
 80002fc:	687b      	ldr	r3, [r7, #4]
}
 80002fe:	4618      	mov	r0, r3
 8000300:	3718      	adds	r7, #24
 8000302:	46bd      	mov	sp, r7
 8000304:	bd80      	pop	{r7, pc}

08000306 <_close>:

int _close(int file)
{
 8000306:	b480      	push	{r7}
 8000308:	b083      	sub	sp, #12
 800030a:	af00      	add	r7, sp, #0
 800030c:	6078      	str	r0, [r7, #4]
	return -1;
 800030e:	f04f 33ff 	mov.w	r3, #4294967295
}
 8000312:	4618      	mov	r0, r3
 8000314:	370c      	adds	r7, #12
 8000316:	46bd      	mov	sp, r7
 8000318:	f85d 7b04 	ldr.w	r7, [sp], #4
 800031c:	4770      	bx	lr

0800031e <_fstat>:


int _fstat(int file, struct stat *st)
{
 800031e:	b480      	push	{r7}
 8000320:	b083      	sub	sp, #12
 8000322:	af00      	add	r7, sp, #0
 8000324:	6078      	str	r0, [r7, #4]
 8000326:	6039      	str	r1, [r7, #0]
	st->st_mode = S_IFCHR;
 8000328:	683b      	ldr	r3, [r7, #0]
 800032a:	f44f 5200 	mov.w	r2, #8192	; 0x2000
 800032e:	605a      	str	r2, [r3, #4]
	return 0;
 8000330:	2300      	movs	r3, #0
}
 8000332:	4618      	mov	r0, r3
 8000334:	370c      	adds	r7, #12
 8000336:	46bd      	mov	sp, r7
 8000338:	f85d 7b04 	ldr.w	r7, [sp], #4
 800033c:	4770      	bx	lr

0800033e <_isatty>:

int _isatty(int file)
{
 800033e:	b480      	push	{r7}
 8000340:	b083      	sub	sp, #12
 8000342:	af00      	add	r7, sp, #0
 8000344:	6078      	str	r0, [r7, #4]
	return 1;
 8000346:	2301      	movs	r3, #1
}
 8000348:	4618      	mov	r0, r3
 800034a:	370c      	adds	r7, #12
 800034c:	46bd      	mov	sp, r7
 800034e:	f85d 7b04 	ldr.w	r7, [sp], #4
 8000352:	4770      	bx	lr

08000354 <_lseek>:

int _lseek(int file, int ptr, int dir)
{
 8000354:	b480      	push	{r7}
 8000356:	b085      	sub	sp, #20
 8000358:	af00      	add	r7, sp, #0
 800035a:	60f8      	str	r0, [r7, #12]
 800035c:	60b9      	str	r1, [r7, #8]
 800035e:	607a      	str	r2, [r7, #4]
	return 0;
 8000360:	2300      	movs	r3, #0
}
 8000362:	4618      	mov	r0, r3
 8000364:	3714      	adds	r7, #20
 8000366:	46bd      	mov	sp, r7
 8000368:	f85d 7b04 	ldr.w	r7, [sp], #4
 800036c:	4770      	bx	lr
	...

08000370 <_sbrk>:
 *
 * @param incr Memory size
 * @return Pointer to allocated memory
 */
void *_sbrk(ptrdiff_t incr)
{
 8000370:	b580      	push	{r7, lr}
 8000372:	b086      	sub	sp, #24
 8000374:	af00      	add	r7, sp, #0
 8000376:	6078      	str	r0, [r7, #4]
  extern uint8_t _end; /* Symbol defined in the linker script */
  extern uint8_t _estack; /* Symbol defined in the linker script */
  extern uint32_t _Min_Stack_Size; /* Symbol defined in the linker script */
  const uint32_t stack_limit = (uint32_t)&_estack - (uint32_t)&_Min_Stack_Size;
 8000378:	4a14      	ldr	r2, [pc, #80]	; (80003cc <_sbrk+0x5c>)
 800037a:	4b15      	ldr	r3, [pc, #84]	; (80003d0 <_sbrk+0x60>)
 800037c:	1ad3      	subs	r3, r2, r3
 800037e:	617b      	str	r3, [r7, #20]
  const uint8_t *max_heap = (uint8_t *)stack_limit;
 8000380:	697b      	ldr	r3, [r7, #20]
 8000382:	613b      	str	r3, [r7, #16]
  uint8_t *prev_heap_end;

  /* Initialize heap end at first call */
  if (NULL == __sbrk_heap_end)
 8000384:	4b13      	ldr	r3, [pc, #76]	; (80003d4 <_sbrk+0x64>)
 8000386:	681b      	ldr	r3, [r3, #0]
 8000388:	2b00      	cmp	r3, #0
 800038a:	d102      	bne.n	8000392 <_sbrk+0x22>
  {
    __sbrk_heap_end = &_end;
 800038c:	4b11      	ldr	r3, [pc, #68]	; (80003d4 <_sbrk+0x64>)
 800038e:	4a12      	ldr	r2, [pc, #72]	; (80003d8 <_sbrk+0x68>)
 8000390:	601a      	str	r2, [r3, #0]
  }

  /* Protect heap from growing into the reserved MSP stack */
  if (__sbrk_heap_end + incr > max_heap)
 8000392:	4b10      	ldr	r3, [pc, #64]	; (80003d4 <_sbrk+0x64>)
 8000394:	681a      	ldr	r2, [r3, #0]
 8000396:	687b      	ldr	r3, [r7, #4]
 8000398:	4413      	add	r3, r2
 800039a:	693a      	ldr	r2, [r7, #16]
 800039c:	429a      	cmp	r2, r3
 800039e:	d207      	bcs.n	80003b0 <_sbrk+0x40>
  {
    errno = ENOMEM;
 80003a0:	f000 f8da 	bl	8000558 <__errno>
 80003a4:	4603      	mov	r3, r0
 80003a6:	220c      	movs	r2, #12
 80003a8:	601a      	str	r2, [r3, #0]
    return (void *)-1;
 80003aa:	f04f 33ff 	mov.w	r3, #4294967295
 80003ae:	e009      	b.n	80003c4 <_sbrk+0x54>
  }

  prev_heap_end = __sbrk_heap_end;
 80003b0:	4b08      	ldr	r3, [pc, #32]	; (80003d4 <_sbrk+0x64>)
 80003b2:	681b      	ldr	r3, [r3, #0]
 80003b4:	60fb      	str	r3, [r7, #12]
  __sbrk_heap_end += incr;
 80003b6:	4b07      	ldr	r3, [pc, #28]	; (80003d4 <_sbrk+0x64>)
 80003b8:	681a      	ldr	r2, [r3, #0]
 80003ba:	687b      	ldr	r3, [r7, #4]
 80003bc:	4413      	add	r3, r2
 80003be:	4a05      	ldr	r2, [pc, #20]	; (80003d4 <_sbrk+0x64>)
 80003c0:	6013      	str	r3, [r2, #0]

  return (void *)prev_heap_end;
 80003c2:	68fb      	ldr	r3, [r7, #12]
}
 80003c4:	4618      	mov	r0, r3
 80003c6:	3718      	adds	r7, #24
 80003c8:	46bd      	mov	sp, r7
 80003ca:	bd80      	pop	{r7, pc}
 80003cc:	20020000 	.word	0x20020000
 80003d0:	00000400 	.word	0x00000400
 80003d4:	20000080 	.word	0x20000080
 80003d8:	200000a0 	.word	0x200000a0

080003dc <__io_putchar>:



void uart2_write(int ch);

int __io_putchar(int ch){
 80003dc:	b580      	push	{r7, lr}
 80003de:	b082      	sub	sp, #8
 80003e0:	af00      	add	r7, sp, #0
 80003e2:	6078      	str	r0, [r7, #4]
	uart2_write(ch);
 80003e4:	6878      	ldr	r0, [r7, #4]
 80003e6:	f000 f84f 	bl	8000488 <uart2_write>
	return ch;
 80003ea:	687b      	ldr	r3, [r7, #4]
}
 80003ec:	4618      	mov	r0, r3
 80003ee:	3708      	adds	r7, #8
 80003f0:	46bd      	mov	sp, r7
 80003f2:	bd80      	pop	{r7, pc}

080003f4 <uart2_tx_init>:

void uart2_tx_init(void){
 80003f4:	b580      	push	{r7, lr}
 80003f6:	af00      	add	r7, sp, #0
	/*********configure the uart gpioa pin*********/
	/*enable clock access to gpioa*/
	RCC->AHB1ENR |= GPIOAEN;
 80003f8:	4b1f      	ldr	r3, [pc, #124]	; (8000478 <uart2_tx_init+0x84>)
 80003fa:	6b1b      	ldr	r3, [r3, #48]	; 0x30
 80003fc:	4a1e      	ldr	r2, [pc, #120]	; (8000478 <uart2_tx_init+0x84>)
 80003fe:	f043 0301 	orr.w	r3, r3, #1
 8000402:	6313      	str	r3, [r2, #48]	; 0x30

	/*set PA2 mode to alternate function mode*/
	GPIOA->MODER &=~ (1U<<4);
 8000404:	4b1d      	ldr	r3, [pc, #116]	; (800047c <uart2_tx_init+0x88>)
 8000406:	681b      	ldr	r3, [r3, #0]
 8000408:	4a1c      	ldr	r2, [pc, #112]	; (800047c <uart2_tx_init+0x88>)
 800040a:	f023 0310 	bic.w	r3, r3, #16
 800040e:	6013      	str	r3, [r2, #0]
	GPIOA->MODER |= (1U<<5);
 8000410:	4b1a      	ldr	r3, [pc, #104]	; (800047c <uart2_tx_init+0x88>)
 8000412:	681b      	ldr	r3, [r3, #0]
 8000414:	4a19      	ldr	r2, [pc, #100]	; (800047c <uart2_tx_init+0x88>)
 8000416:	f043 0320 	orr.w	r3, r3, #32
 800041a:	6013      	str	r3, [r2, #0]

	/*set PA2 alternate function type to UART_TX (AF07)*/
	GPIOA->AFR[0] |= (1U<<8);
 800041c:	4b17      	ldr	r3, [pc, #92]	; (800047c <uart2_tx_init+0x88>)
 800041e:	6a1b      	ldr	r3, [r3, #32]
 8000420:	4a16      	ldr	r2, [pc, #88]	; (800047c <uart2_tx_init+0x88>)
 8000422:	f443 7380 	orr.w	r3, r3, #256	; 0x100
 8000426:	6213      	str	r3, [r2, #32]
	GPIOA->AFR[0] |= (1U<<9);
 8000428:	4b14      	ldr	r3, [pc, #80]	; (800047c <uart2_tx_init+0x88>)
 800042a:	6a1b      	ldr	r3, [r3, #32]
 800042c:	4a13      	ldr	r2, [pc, #76]	; (800047c <uart2_tx_init+0x88>)
 800042e:	f443 7300 	orr.w	r3, r3, #512	; 0x200
 8000432:	6213      	str	r3, [r2, #32]
	GPIOA->AFR[0] |= (1U<<10);
 8000434:	4b11      	ldr	r3, [pc, #68]	; (800047c <uart2_tx_init+0x88>)
 8000436:	6a1b      	ldr	r3, [r3, #32]
 8000438:	4a10      	ldr	r2, [pc, #64]	; (800047c <uart2_tx_init+0x88>)
 800043a:	f443 6380 	orr.w	r3, r3, #1024	; 0x400
 800043e:	6213      	str	r3, [r2, #32]
	GPIOA->AFR[0] &=~ (1U<<11);
 8000440:	4b0e      	ldr	r3, [pc, #56]	; (800047c <uart2_tx_init+0x88>)
 8000442:	6a1b      	ldr	r3, [r3, #32]
 8000444:	4a0d      	ldr	r2, [pc, #52]	; (800047c <uart2_tx_init+0x88>)
 8000446:	f423 6300 	bic.w	r3, r3, #2048	; 0x800
 800044a:	6213      	str	r3, [r2, #32]

	/*********configure the uart module *********/
	/*enable clock access to uart2*/
	RCC->APB1ENR |= UART2EN;
 800044c:	4b0a      	ldr	r3, [pc, #40]	; (8000478 <uart2_tx_init+0x84>)
 800044e:	6c1b      	ldr	r3, [r3, #64]	; 0x40
 8000450:	4a09      	ldr	r2, [pc, #36]	; (8000478 <uart2_tx_init+0x84>)
 8000452:	f443 3300 	orr.w	r3, r3, #131072	; 0x20000
 8000456:	6413      	str	r3, [r2, #64]	; 0x40

	/*configure baudrate*/
	uart_set_baudrate(USART2,APB1_CLK,UART_BAUDRATE);
 8000458:	f44f 32e1 	mov.w	r2, #115200	; 0x1c200
 800045c:	4908      	ldr	r1, [pc, #32]	; (8000480 <uart2_tx_init+0x8c>)
 800045e:	4809      	ldr	r0, [pc, #36]	; (8000484 <uart2_tx_init+0x90>)
 8000460:	f000 f82a 	bl	80004b8 <uart_set_baudrate>

	/*configure the transfer direction*/
	USART2 ->CR1 = CR1_TE;
 8000464:	4b07      	ldr	r3, [pc, #28]	; (8000484 <uart2_tx_init+0x90>)
 8000466:	2208      	movs	r2, #8
 8000468:	60da      	str	r2, [r3, #12]

	/*enable uart module*/
	USART2 ->CR1 = CR1_UE;
 800046a:	4b06      	ldr	r3, [pc, #24]	; (8000484 <uart2_tx_init+0x90>)
 800046c:	f44f 5200 	mov.w	r2, #8192	; 0x2000
 8000470:	60da      	str	r2, [r3, #12]

}
 8000472:	bf00      	nop
 8000474:	bd80      	pop	{r7, pc}
 8000476:	bf00      	nop
 8000478:	40023800 	.word	0x40023800
 800047c:	40020000 	.word	0x40020000
 8000480:	00f42400 	.word	0x00f42400
 8000484:	40004400 	.word	0x40004400

08000488 <uart2_write>:

void uart2_write(int ch){
 8000488:	b480      	push	{r7}
 800048a:	b083      	sub	sp, #12
 800048c:	af00      	add	r7, sp, #0
 800048e:	6078      	str	r0, [r7, #4]
	/*make sure the transmit data register is empty*/
	while(!(USART2->SR & SR_TXE)){}
 8000490:	bf00      	nop
 8000492:	4b08      	ldr	r3, [pc, #32]	; (80004b4 <uart2_write+0x2c>)
 8000494:	681b      	ldr	r3, [r3, #0]
 8000496:	f003 0380 	and.w	r3, r3, #128	; 0x80
 800049a:	2b00      	cmp	r3, #0
 800049c:	d0f9      	beq.n	8000492 <uart2_write+0xa>
	/*write to transmit data register*/
	USART2->DR = (ch & 0xFF);
 800049e:	687b      	ldr	r3, [r7, #4]
 80004a0:	4a04      	ldr	r2, [pc, #16]	; (80004b4 <uart2_write+0x2c>)
 80004a2:	b2db      	uxtb	r3, r3
 80004a4:	6053      	str	r3, [r2, #4]
}
 80004a6:	bf00      	nop
 80004a8:	370c      	adds	r7, #12
 80004aa:	46bd      	mov	sp, r7
 80004ac:	f85d 7b04 	ldr.w	r7, [sp], #4
 80004b0:	4770      	bx	lr
 80004b2:	bf00      	nop
 80004b4:	40004400 	.word	0x40004400

080004b8 <uart_set_baudrate>:

static void uart_set_baudrate(USART_TypeDef *USARTx, uint32_t PeriphClk, uint32_t BaudRate){
 80004b8:	b580      	push	{r7, lr}
 80004ba:	b084      	sub	sp, #16
 80004bc:	af00      	add	r7, sp, #0
 80004be:	60f8      	str	r0, [r7, #12]
 80004c0:	60b9      	str	r1, [r7, #8]
 80004c2:	607a      	str	r2, [r7, #4]
	USARTx->BRR = compute_uart_bd(PeriphClk, BaudRate);
 80004c4:	6879      	ldr	r1, [r7, #4]
 80004c6:	68b8      	ldr	r0, [r7, #8]
 80004c8:	f000 f808 	bl	80004dc <compute_uart_bd>
 80004cc:	4603      	mov	r3, r0
 80004ce:	461a      	mov	r2, r3
 80004d0:	68fb      	ldr	r3, [r7, #12]
 80004d2:	609a      	str	r2, [r3, #8]
}
 80004d4:	bf00      	nop
 80004d6:	3710      	adds	r7, #16
 80004d8:	46bd      	mov	sp, r7
 80004da:	bd80      	pop	{r7, pc}

080004dc <compute_uart_bd>:

static uint16_t compute_uart_bd(uint32_t PeriphClk, uint32_t BaudRate){
 80004dc:	b480      	push	{r7}
 80004de:	b083      	sub	sp, #12
 80004e0:	af00      	add	r7, sp, #0
 80004e2:	6078      	str	r0, [r7, #4]
 80004e4:	6039      	str	r1, [r7, #0]
	return ((PeriphClk + (BaudRate/2U))/BaudRate);
 80004e6:	683b      	ldr	r3, [r7, #0]
 80004e8:	085a      	lsrs	r2, r3, #1
 80004ea:	687b      	ldr	r3, [r7, #4]
 80004ec:	441a      	add	r2, r3
 80004ee:	683b      	ldr	r3, [r7, #0]
 80004f0:	fbb2 f3f3 	udiv	r3, r2, r3
 80004f4:	b29b      	uxth	r3, r3
}
 80004f6:	4618      	mov	r0, r3
 80004f8:	370c      	adds	r7, #12
 80004fa:	46bd      	mov	sp, r7
 80004fc:	f85d 7b04 	ldr.w	r7, [sp], #4
 8000500:	4770      	bx	lr
	...

08000504 <Reset_Handler>:

  .section .text.Reset_Handler
  .weak Reset_Handler
  .type Reset_Handler, %function
Reset_Handler:
  ldr   r0, =_estack
 8000504:	480d      	ldr	r0, [pc, #52]	; (800053c <LoopForever+0x2>)
  mov   sp, r0          /* set stack pointer */
 8000506:	4685      	mov	sp, r0
/* Call the clock system intitialization function.*/
  bl  SystemInit
 8000508:	f3af 8000 	nop.w

/* Copy the data segment initializers from flash to SRAM */
  ldr r0, =_sdata
 800050c:	480c      	ldr	r0, [pc, #48]	; (8000540 <LoopForever+0x6>)
  ldr r1, =_edata
 800050e:	490d      	ldr	r1, [pc, #52]	; (8000544 <LoopForever+0xa>)
  ldr r2, =_sidata
 8000510:	4a0d      	ldr	r2, [pc, #52]	; (8000548 <LoopForever+0xe>)
  movs r3, #0
 8000512:	2300      	movs	r3, #0
  b LoopCopyDataInit
 8000514:	e002      	b.n	800051c <LoopCopyDataInit>

08000516 <CopyDataInit>:

CopyDataInit:
  ldr r4, [r2, r3]
 8000516:	58d4      	ldr	r4, [r2, r3]
  str r4, [r0, r3]
 8000518:	50c4      	str	r4, [r0, r3]
  adds r3, r3, #4
 800051a:	3304      	adds	r3, #4

0800051c <LoopCopyDataInit>:

LoopCopyDataInit:
  adds r4, r0, r3
 800051c:	18c4      	adds	r4, r0, r3
  cmp r4, r1
 800051e:	428c      	cmp	r4, r1
  bcc CopyDataInit
 8000520:	d3f9      	bcc.n	8000516 <CopyDataInit>

/* Zero fill the bss segment. */
  ldr r2, =_sbss
 8000522:	4a0a      	ldr	r2, [pc, #40]	; (800054c <LoopForever+0x12>)
  ldr r4, =_ebss
 8000524:	4c0a      	ldr	r4, [pc, #40]	; (8000550 <LoopForever+0x16>)
  movs r3, #0
 8000526:	2300      	movs	r3, #0
  b LoopFillZerobss
 8000528:	e001      	b.n	800052e <LoopFillZerobss>

0800052a <FillZerobss>:

FillZerobss:
  str  r3, [r2]
 800052a:	6013      	str	r3, [r2, #0]
  adds r2, r2, #4
 800052c:	3204      	adds	r2, #4

0800052e <LoopFillZerobss>:

LoopFillZerobss:
  cmp r2, r4
 800052e:	42a2      	cmp	r2, r4
  bcc FillZerobss
 8000530:	d3fb      	bcc.n	800052a <FillZerobss>

/* Call static constructors */
  bl __libc_init_array
 8000532:	f000 f817 	bl	8000564 <__libc_init_array>
/* Call the application's entry point.*/
  bl main
 8000536:	f7ff fea3 	bl	8000280 <main>

0800053a <LoopForever>:

LoopForever:
    b LoopForever
 800053a:	e7fe      	b.n	800053a <LoopForever>
  ldr   r0, =_estack
 800053c:	20020000 	.word	0x20020000
  ldr r0, =_sdata
 8000540:	20000000 	.word	0x20000000
  ldr r1, =_edata
 8000544:	20000064 	.word	0x20000064
  ldr r2, =_sidata
 8000548:	0800152c 	.word	0x0800152c
  ldr r2, =_sbss
 800054c:	20000064 	.word	0x20000064
  ldr r4, =_ebss
 8000550:	2000009c 	.word	0x2000009c

08000554 <ADC_IRQHandler>:
 * @retval : None
*/
  .section .text.Default_Handler,"ax",%progbits
Default_Handler:
Infinite_Loop:
  b Infinite_Loop
 8000554:	e7fe      	b.n	8000554 <ADC_IRQHandler>
	...

08000558 <__errno>:
 8000558:	4b01      	ldr	r3, [pc, #4]	; (8000560 <__errno+0x8>)
 800055a:	6818      	ldr	r0, [r3, #0]
 800055c:	4770      	bx	lr
 800055e:	bf00      	nop
 8000560:	20000000 	.word	0x20000000

08000564 <__libc_init_array>:
 8000564:	b570      	push	{r4, r5, r6, lr}
 8000566:	4d0d      	ldr	r5, [pc, #52]	; (800059c <__libc_init_array+0x38>)
 8000568:	4c0d      	ldr	r4, [pc, #52]	; (80005a0 <__libc_init_array+0x3c>)
 800056a:	1b64      	subs	r4, r4, r5
 800056c:	10a4      	asrs	r4, r4, #2
 800056e:	2600      	movs	r6, #0
 8000570:	42a6      	cmp	r6, r4
 8000572:	d109      	bne.n	8000588 <__libc_init_array+0x24>
 8000574:	4d0b      	ldr	r5, [pc, #44]	; (80005a4 <__libc_init_array+0x40>)
 8000576:	4c0c      	ldr	r4, [pc, #48]	; (80005a8 <__libc_init_array+0x44>)
 8000578:	f000 ff76 	bl	8001468 <_init>
 800057c:	1b64      	subs	r4, r4, r5
 800057e:	10a4      	asrs	r4, r4, #2
 8000580:	2600      	movs	r6, #0
 8000582:	42a6      	cmp	r6, r4
 8000584:	d105      	bne.n	8000592 <__libc_init_array+0x2e>
 8000586:	bd70      	pop	{r4, r5, r6, pc}
 8000588:	f855 3b04 	ldr.w	r3, [r5], #4
 800058c:	4798      	blx	r3
 800058e:	3601      	adds	r6, #1
 8000590:	e7ee      	b.n	8000570 <__libc_init_array+0xc>
 8000592:	f855 3b04 	ldr.w	r3, [r5], #4
 8000596:	4798      	blx	r3
 8000598:	3601      	adds	r6, #1
 800059a:	e7f2      	b.n	8000582 <__libc_init_array+0x1e>
 800059c:	08001524 	.word	0x08001524
 80005a0:	08001524 	.word	0x08001524
 80005a4:	08001524 	.word	0x08001524
 80005a8:	08001528 	.word	0x08001528

080005ac <memset>:
 80005ac:	4402      	add	r2, r0
 80005ae:	4603      	mov	r3, r0
 80005b0:	4293      	cmp	r3, r2
 80005b2:	d100      	bne.n	80005b6 <memset+0xa>
 80005b4:	4770      	bx	lr
 80005b6:	f803 1b01 	strb.w	r1, [r3], #1
 80005ba:	e7f9      	b.n	80005b0 <memset+0x4>

080005bc <iprintf>:
 80005bc:	b40f      	push	{r0, r1, r2, r3}
 80005be:	4b0a      	ldr	r3, [pc, #40]	; (80005e8 <iprintf+0x2c>)
 80005c0:	b513      	push	{r0, r1, r4, lr}
 80005c2:	681c      	ldr	r4, [r3, #0]
 80005c4:	b124      	cbz	r4, 80005d0 <iprintf+0x14>
 80005c6:	69a3      	ldr	r3, [r4, #24]
 80005c8:	b913      	cbnz	r3, 80005d0 <iprintf+0x14>
 80005ca:	4620      	mov	r0, r4
 80005cc:	f000 f866 	bl	800069c <__sinit>
 80005d0:	ab05      	add	r3, sp, #20
 80005d2:	9a04      	ldr	r2, [sp, #16]
 80005d4:	68a1      	ldr	r1, [r4, #8]
 80005d6:	9301      	str	r3, [sp, #4]
 80005d8:	4620      	mov	r0, r4
 80005da:	f000 f983 	bl	80008e4 <_vfiprintf_r>
 80005de:	b002      	add	sp, #8
 80005e0:	e8bd 4010 	ldmia.w	sp!, {r4, lr}
 80005e4:	b004      	add	sp, #16
 80005e6:	4770      	bx	lr
 80005e8:	20000000 	.word	0x20000000

080005ec <std>:
 80005ec:	2300      	movs	r3, #0
 80005ee:	b510      	push	{r4, lr}
 80005f0:	4604      	mov	r4, r0
 80005f2:	e9c0 3300 	strd	r3, r3, [r0]
 80005f6:	e9c0 3304 	strd	r3, r3, [r0, #16]
 80005fa:	6083      	str	r3, [r0, #8]
 80005fc:	8181      	strh	r1, [r0, #12]
 80005fe:	6643      	str	r3, [r0, #100]	; 0x64
 8000600:	81c2      	strh	r2, [r0, #14]
 8000602:	6183      	str	r3, [r0, #24]
 8000604:	4619      	mov	r1, r3
 8000606:	2208      	movs	r2, #8
 8000608:	305c      	adds	r0, #92	; 0x5c
 800060a:	f7ff ffcf 	bl	80005ac <memset>
 800060e:	4b05      	ldr	r3, [pc, #20]	; (8000624 <std+0x38>)
 8000610:	6263      	str	r3, [r4, #36]	; 0x24
 8000612:	4b05      	ldr	r3, [pc, #20]	; (8000628 <std+0x3c>)
 8000614:	62a3      	str	r3, [r4, #40]	; 0x28
 8000616:	4b05      	ldr	r3, [pc, #20]	; (800062c <std+0x40>)
 8000618:	62e3      	str	r3, [r4, #44]	; 0x2c
 800061a:	4b05      	ldr	r3, [pc, #20]	; (8000630 <std+0x44>)
 800061c:	6224      	str	r4, [r4, #32]
 800061e:	6323      	str	r3, [r4, #48]	; 0x30
 8000620:	bd10      	pop	{r4, pc}
 8000622:	bf00      	nop
 8000624:	08000e8d 	.word	0x08000e8d
 8000628:	08000eaf 	.word	0x08000eaf
 800062c:	08000ee7 	.word	0x08000ee7
 8000630:	08000f0b 	.word	0x08000f0b

08000634 <_cleanup_r>:
 8000634:	4901      	ldr	r1, [pc, #4]	; (800063c <_cleanup_r+0x8>)
 8000636:	f000 b8af 	b.w	8000798 <_fwalk_reent>
 800063a:	bf00      	nop
 800063c:	080011e5 	.word	0x080011e5

08000640 <__sfmoreglue>:
 8000640:	b570      	push	{r4, r5, r6, lr}
 8000642:	1e4a      	subs	r2, r1, #1
 8000644:	2568      	movs	r5, #104	; 0x68
 8000646:	4355      	muls	r5, r2
 8000648:	460e      	mov	r6, r1
 800064a:	f105 0174 	add.w	r1, r5, #116	; 0x74
 800064e:	f000 f8c5 	bl	80007dc <_malloc_r>
 8000652:	4604      	mov	r4, r0
 8000654:	b140      	cbz	r0, 8000668 <__sfmoreglue+0x28>
 8000656:	2100      	movs	r1, #0
 8000658:	e9c0 1600 	strd	r1, r6, [r0]
 800065c:	300c      	adds	r0, #12
 800065e:	60a0      	str	r0, [r4, #8]
 8000660:	f105 0268 	add.w	r2, r5, #104	; 0x68
 8000664:	f7ff ffa2 	bl	80005ac <memset>
 8000668:	4620      	mov	r0, r4
 800066a:	bd70      	pop	{r4, r5, r6, pc}

0800066c <__sfp_lock_acquire>:
 800066c:	4801      	ldr	r0, [pc, #4]	; (8000674 <__sfp_lock_acquire+0x8>)
 800066e:	f000 b8b3 	b.w	80007d8 <__retarget_lock_acquire_recursive>
 8000672:	bf00      	nop
 8000674:	20000094 	.word	0x20000094

08000678 <__sfp_lock_release>:
 8000678:	4801      	ldr	r0, [pc, #4]	; (8000680 <__sfp_lock_release+0x8>)
 800067a:	f000 b8ae 	b.w	80007da <__retarget_lock_release_recursive>
 800067e:	bf00      	nop
 8000680:	20000094 	.word	0x20000094

08000684 <__sinit_lock_acquire>:
 8000684:	4801      	ldr	r0, [pc, #4]	; (800068c <__sinit_lock_acquire+0x8>)
 8000686:	f000 b8a7 	b.w	80007d8 <__retarget_lock_acquire_recursive>
 800068a:	bf00      	nop
 800068c:	2000008f 	.word	0x2000008f

08000690 <__sinit_lock_release>:
 8000690:	4801      	ldr	r0, [pc, #4]	; (8000698 <__sinit_lock_release+0x8>)
 8000692:	f000 b8a2 	b.w	80007da <__retarget_lock_release_recursive>
 8000696:	bf00      	nop
 8000698:	2000008f 	.word	0x2000008f

0800069c <__sinit>:
 800069c:	b510      	push	{r4, lr}
 800069e:	4604      	mov	r4, r0
 80006a0:	f7ff fff0 	bl	8000684 <__sinit_lock_acquire>
 80006a4:	69a3      	ldr	r3, [r4, #24]
 80006a6:	b11b      	cbz	r3, 80006b0 <__sinit+0x14>
 80006a8:	e8bd 4010 	ldmia.w	sp!, {r4, lr}
 80006ac:	f7ff bff0 	b.w	8000690 <__sinit_lock_release>
 80006b0:	e9c4 3312 	strd	r3, r3, [r4, #72]	; 0x48
 80006b4:	6523      	str	r3, [r4, #80]	; 0x50
 80006b6:	4b13      	ldr	r3, [pc, #76]	; (8000704 <__sinit+0x68>)
 80006b8:	4a13      	ldr	r2, [pc, #76]	; (8000708 <__sinit+0x6c>)
 80006ba:	681b      	ldr	r3, [r3, #0]
 80006bc:	62a2      	str	r2, [r4, #40]	; 0x28
 80006be:	42a3      	cmp	r3, r4
 80006c0:	bf04      	itt	eq
 80006c2:	2301      	moveq	r3, #1
 80006c4:	61a3      	streq	r3, [r4, #24]
 80006c6:	4620      	mov	r0, r4
 80006c8:	f000 f820 	bl	800070c <__sfp>
 80006cc:	6060      	str	r0, [r4, #4]
 80006ce:	4620      	mov	r0, r4
 80006d0:	f000 f81c 	bl	800070c <__sfp>
 80006d4:	60a0      	str	r0, [r4, #8]
 80006d6:	4620      	mov	r0, r4
 80006d8:	f000 f818 	bl	800070c <__sfp>
 80006dc:	2200      	movs	r2, #0
 80006de:	60e0      	str	r0, [r4, #12]
 80006e0:	2104      	movs	r1, #4
 80006e2:	6860      	ldr	r0, [r4, #4]
 80006e4:	f7ff ff82 	bl	80005ec <std>
 80006e8:	68a0      	ldr	r0, [r4, #8]
 80006ea:	2201      	movs	r2, #1
 80006ec:	2109      	movs	r1, #9
 80006ee:	f7ff ff7d 	bl	80005ec <std>
 80006f2:	68e0      	ldr	r0, [r4, #12]
 80006f4:	2202      	movs	r2, #2
 80006f6:	2112      	movs	r1, #18
 80006f8:	f7ff ff78 	bl	80005ec <std>
 80006fc:	2301      	movs	r3, #1
 80006fe:	61a3      	str	r3, [r4, #24]
 8000700:	e7d2      	b.n	80006a8 <__sinit+0xc>
 8000702:	bf00      	nop
 8000704:	0800148c 	.word	0x0800148c
 8000708:	08000635 	.word	0x08000635

0800070c <__sfp>:
 800070c:	b5f8      	push	{r3, r4, r5, r6, r7, lr}
 800070e:	4607      	mov	r7, r0
 8000710:	f7ff ffac 	bl	800066c <__sfp_lock_acquire>
 8000714:	4b1e      	ldr	r3, [pc, #120]	; (8000790 <__sfp+0x84>)
 8000716:	681e      	ldr	r6, [r3, #0]
 8000718:	69b3      	ldr	r3, [r6, #24]
 800071a:	b913      	cbnz	r3, 8000722 <__sfp+0x16>
 800071c:	4630      	mov	r0, r6
 800071e:	f7ff ffbd 	bl	800069c <__sinit>
 8000722:	3648      	adds	r6, #72	; 0x48
 8000724:	e9d6 3401 	ldrd	r3, r4, [r6, #4]
 8000728:	3b01      	subs	r3, #1
 800072a:	d503      	bpl.n	8000734 <__sfp+0x28>
 800072c:	6833      	ldr	r3, [r6, #0]
 800072e:	b30b      	cbz	r3, 8000774 <__sfp+0x68>
 8000730:	6836      	ldr	r6, [r6, #0]
 8000732:	e7f7      	b.n	8000724 <__sfp+0x18>
 8000734:	f9b4 500c 	ldrsh.w	r5, [r4, #12]
 8000738:	b9d5      	cbnz	r5, 8000770 <__sfp+0x64>
 800073a:	4b16      	ldr	r3, [pc, #88]	; (8000794 <__sfp+0x88>)
 800073c:	60e3      	str	r3, [r4, #12]
 800073e:	f104 0058 	add.w	r0, r4, #88	; 0x58
 8000742:	6665      	str	r5, [r4, #100]	; 0x64
 8000744:	f000 f847 	bl	80007d6 <__retarget_lock_init_recursive>
 8000748:	f7ff ff96 	bl	8000678 <__sfp_lock_release>
 800074c:	e9c4 5501 	strd	r5, r5, [r4, #4]
 8000750:	e9c4 5504 	strd	r5, r5, [r4, #16]
 8000754:	6025      	str	r5, [r4, #0]
 8000756:	61a5      	str	r5, [r4, #24]
 8000758:	2208      	movs	r2, #8
 800075a:	4629      	mov	r1, r5
 800075c:	f104 005c 	add.w	r0, r4, #92	; 0x5c
 8000760:	f7ff ff24 	bl	80005ac <memset>
 8000764:	e9c4 550d 	strd	r5, r5, [r4, #52]	; 0x34
 8000768:	e9c4 5512 	strd	r5, r5, [r4, #72]	; 0x48
 800076c:	4620      	mov	r0, r4
 800076e:	bdf8      	pop	{r3, r4, r5, r6, r7, pc}
 8000770:	3468      	adds	r4, #104	; 0x68
 8000772:	e7d9      	b.n	8000728 <__sfp+0x1c>
 8000774:	2104      	movs	r1, #4
 8000776:	4638      	mov	r0, r7
 8000778:	f7ff ff62 	bl	8000640 <__sfmoreglue>
 800077c:	4604      	mov	r4, r0
 800077e:	6030      	str	r0, [r6, #0]
 8000780:	2800      	cmp	r0, #0
 8000782:	d1d5      	bne.n	8000730 <__sfp+0x24>
 8000784:	f7ff ff78 	bl	8000678 <__sfp_lock_release>
 8000788:	230c      	movs	r3, #12
 800078a:	603b      	str	r3, [r7, #0]
 800078c:	e7ee      	b.n	800076c <__sfp+0x60>
 800078e:	bf00      	nop
 8000790:	0800148c 	.word	0x0800148c
 8000794:	ffff0001 	.word	0xffff0001

08000798 <_fwalk_reent>:
 8000798:	e92d 43f8 	stmdb	sp!, {r3, r4, r5, r6, r7, r8, r9, lr}
 800079c:	4606      	mov	r6, r0
 800079e:	4688      	mov	r8, r1
 80007a0:	f100 0448 	add.w	r4, r0, #72	; 0x48
 80007a4:	2700      	movs	r7, #0
 80007a6:	e9d4 9501 	ldrd	r9, r5, [r4, #4]
 80007aa:	f1b9 0901 	subs.w	r9, r9, #1
 80007ae:	d505      	bpl.n	80007bc <_fwalk_reent+0x24>
 80007b0:	6824      	ldr	r4, [r4, #0]
 80007b2:	2c00      	cmp	r4, #0
 80007b4:	d1f7      	bne.n	80007a6 <_fwalk_reent+0xe>
 80007b6:	4638      	mov	r0, r7
 80007b8:	e8bd 83f8 	ldmia.w	sp!, {r3, r4, r5, r6, r7, r8, r9, pc}
 80007bc:	89ab      	ldrh	r3, [r5, #12]
 80007be:	2b01      	cmp	r3, #1
 80007c0:	d907      	bls.n	80007d2 <_fwalk_reent+0x3a>
 80007c2:	f9b5 300e 	ldrsh.w	r3, [r5, #14]
 80007c6:	3301      	adds	r3, #1
 80007c8:	d003      	beq.n	80007d2 <_fwalk_reent+0x3a>
 80007ca:	4629      	mov	r1, r5
 80007cc:	4630      	mov	r0, r6
 80007ce:	47c0      	blx	r8
 80007d0:	4307      	orrs	r7, r0
 80007d2:	3568      	adds	r5, #104	; 0x68
 80007d4:	e7e9      	b.n	80007aa <_fwalk_reent+0x12>

080007d6 <__retarget_lock_init_recursive>:
 80007d6:	4770      	bx	lr

080007d8 <__retarget_lock_acquire_recursive>:
 80007d8:	4770      	bx	lr

080007da <__retarget_lock_release_recursive>:
 80007da:	4770      	bx	lr

080007dc <_malloc_r>:
 80007dc:	b5f8      	push	{r3, r4, r5, r6, r7, lr}
 80007de:	1ccd      	adds	r5, r1, #3
 80007e0:	f025 0503 	bic.w	r5, r5, #3
 80007e4:	3508      	adds	r5, #8
 80007e6:	2d0c      	cmp	r5, #12
 80007e8:	bf38      	it	cc
 80007ea:	250c      	movcc	r5, #12
 80007ec:	2d00      	cmp	r5, #0
 80007ee:	4606      	mov	r6, r0
 80007f0:	db01      	blt.n	80007f6 <_malloc_r+0x1a>
 80007f2:	42a9      	cmp	r1, r5
 80007f4:	d903      	bls.n	80007fe <_malloc_r+0x22>
 80007f6:	230c      	movs	r3, #12
 80007f8:	6033      	str	r3, [r6, #0]
 80007fa:	2000      	movs	r0, #0
 80007fc:	bdf8      	pop	{r3, r4, r5, r6, r7, pc}
 80007fe:	f000 fda3 	bl	8001348 <__malloc_lock>
 8000802:	4921      	ldr	r1, [pc, #132]	; (8000888 <_malloc_r+0xac>)
 8000804:	680a      	ldr	r2, [r1, #0]
 8000806:	4614      	mov	r4, r2
 8000808:	b99c      	cbnz	r4, 8000832 <_malloc_r+0x56>
 800080a:	4f20      	ldr	r7, [pc, #128]	; (800088c <_malloc_r+0xb0>)
 800080c:	683b      	ldr	r3, [r7, #0]
 800080e:	b923      	cbnz	r3, 800081a <_malloc_r+0x3e>
 8000810:	4621      	mov	r1, r4
 8000812:	4630      	mov	r0, r6
 8000814:	f000 fb2a 	bl	8000e6c <_sbrk_r>
 8000818:	6038      	str	r0, [r7, #0]
 800081a:	4629      	mov	r1, r5
 800081c:	4630      	mov	r0, r6
 800081e:	f000 fb25 	bl	8000e6c <_sbrk_r>
 8000822:	1c43      	adds	r3, r0, #1
 8000824:	d123      	bne.n	800086e <_malloc_r+0x92>
 8000826:	230c      	movs	r3, #12
 8000828:	6033      	str	r3, [r6, #0]
 800082a:	4630      	mov	r0, r6
 800082c:	f000 fd92 	bl	8001354 <__malloc_unlock>
 8000830:	e7e3      	b.n	80007fa <_malloc_r+0x1e>
 8000832:	6823      	ldr	r3, [r4, #0]
 8000834:	1b5b      	subs	r3, r3, r5
 8000836:	d417      	bmi.n	8000868 <_malloc_r+0x8c>
 8000838:	2b0b      	cmp	r3, #11
 800083a:	d903      	bls.n	8000844 <_malloc_r+0x68>
 800083c:	6023      	str	r3, [r4, #0]
 800083e:	441c      	add	r4, r3
 8000840:	6025      	str	r5, [r4, #0]
 8000842:	e004      	b.n	800084e <_malloc_r+0x72>
 8000844:	6863      	ldr	r3, [r4, #4]
 8000846:	42a2      	cmp	r2, r4
 8000848:	bf0c      	ite	eq
 800084a:	600b      	streq	r3, [r1, #0]
 800084c:	6053      	strne	r3, [r2, #4]
 800084e:	4630      	mov	r0, r6
 8000850:	f000 fd80 	bl	8001354 <__malloc_unlock>
 8000854:	f104 000b 	add.w	r0, r4, #11
 8000858:	1d23      	adds	r3, r4, #4
 800085a:	f020 0007 	bic.w	r0, r0, #7
 800085e:	1ac2      	subs	r2, r0, r3
 8000860:	d0cc      	beq.n	80007fc <_malloc_r+0x20>
 8000862:	1a1b      	subs	r3, r3, r0
 8000864:	50a3      	str	r3, [r4, r2]
 8000866:	e7c9      	b.n	80007fc <_malloc_r+0x20>
 8000868:	4622      	mov	r2, r4
 800086a:	6864      	ldr	r4, [r4, #4]
 800086c:	e7cc      	b.n	8000808 <_malloc_r+0x2c>
 800086e:	1cc4      	adds	r4, r0, #3
 8000870:	f024 0403 	bic.w	r4, r4, #3
 8000874:	42a0      	cmp	r0, r4
 8000876:	d0e3      	beq.n	8000840 <_malloc_r+0x64>
 8000878:	1a21      	subs	r1, r4, r0
 800087a:	4630      	mov	r0, r6
 800087c:	f000 faf6 	bl	8000e6c <_sbrk_r>
 8000880:	3001      	adds	r0, #1
 8000882:	d1dd      	bne.n	8000840 <_malloc_r+0x64>
 8000884:	e7cf      	b.n	8000826 <_malloc_r+0x4a>
 8000886:	bf00      	nop
 8000888:	20000084 	.word	0x20000084
 800088c:	20000088 	.word	0x20000088

08000890 <__sfputc_r>:
 8000890:	6893      	ldr	r3, [r2, #8]
 8000892:	3b01      	subs	r3, #1
 8000894:	2b00      	cmp	r3, #0
 8000896:	b410      	push	{r4}
 8000898:	6093      	str	r3, [r2, #8]
 800089a:	da08      	bge.n	80008ae <__sfputc_r+0x1e>
 800089c:	6994      	ldr	r4, [r2, #24]
 800089e:	42a3      	cmp	r3, r4
 80008a0:	db01      	blt.n	80008a6 <__sfputc_r+0x16>
 80008a2:	290a      	cmp	r1, #10
 80008a4:	d103      	bne.n	80008ae <__sfputc_r+0x1e>
 80008a6:	f85d 4b04 	ldr.w	r4, [sp], #4
 80008aa:	f000 bb33 	b.w	8000f14 <__swbuf_r>
 80008ae:	6813      	ldr	r3, [r2, #0]
 80008b0:	1c58      	adds	r0, r3, #1
 80008b2:	6010      	str	r0, [r2, #0]
 80008b4:	7019      	strb	r1, [r3, #0]
 80008b6:	4608      	mov	r0, r1
 80008b8:	f85d 4b04 	ldr.w	r4, [sp], #4
 80008bc:	4770      	bx	lr

080008be <__sfputs_r>:
 80008be:	b5f8      	push	{r3, r4, r5, r6, r7, lr}
 80008c0:	4606      	mov	r6, r0
 80008c2:	460f      	mov	r7, r1
 80008c4:	4614      	mov	r4, r2
 80008c6:	18d5      	adds	r5, r2, r3
 80008c8:	42ac      	cmp	r4, r5
 80008ca:	d101      	bne.n	80008d0 <__sfputs_r+0x12>
 80008cc:	2000      	movs	r0, #0
 80008ce:	e007      	b.n	80008e0 <__sfputs_r+0x22>
 80008d0:	f814 1b01 	ldrb.w	r1, [r4], #1
 80008d4:	463a      	mov	r2, r7
 80008d6:	4630      	mov	r0, r6
 80008d8:	f7ff ffda 	bl	8000890 <__sfputc_r>
 80008dc:	1c43      	adds	r3, r0, #1
 80008de:	d1f3      	bne.n	80008c8 <__sfputs_r+0xa>
 80008e0:	bdf8      	pop	{r3, r4, r5, r6, r7, pc}
	...

080008e4 <_vfiprintf_r>:
 80008e4:	e92d 4ff0 	stmdb	sp!, {r4, r5, r6, r7, r8, r9, sl, fp, lr}
 80008e8:	460d      	mov	r5, r1
 80008ea:	b09d      	sub	sp, #116	; 0x74
 80008ec:	4614      	mov	r4, r2
 80008ee:	4698      	mov	r8, r3
 80008f0:	4606      	mov	r6, r0
 80008f2:	b118      	cbz	r0, 80008fc <_vfiprintf_r+0x18>
 80008f4:	6983      	ldr	r3, [r0, #24]
 80008f6:	b90b      	cbnz	r3, 80008fc <_vfiprintf_r+0x18>
 80008f8:	f7ff fed0 	bl	800069c <__sinit>
 80008fc:	4b89      	ldr	r3, [pc, #548]	; (8000b24 <_vfiprintf_r+0x240>)
 80008fe:	429d      	cmp	r5, r3
 8000900:	d11b      	bne.n	800093a <_vfiprintf_r+0x56>
 8000902:	6875      	ldr	r5, [r6, #4]
 8000904:	6e6b      	ldr	r3, [r5, #100]	; 0x64
 8000906:	07d9      	lsls	r1, r3, #31
 8000908:	d405      	bmi.n	8000916 <_vfiprintf_r+0x32>
 800090a:	89ab      	ldrh	r3, [r5, #12]
 800090c:	059a      	lsls	r2, r3, #22
 800090e:	d402      	bmi.n	8000916 <_vfiprintf_r+0x32>
 8000910:	6da8      	ldr	r0, [r5, #88]	; 0x58
 8000912:	f7ff ff61 	bl	80007d8 <__retarget_lock_acquire_recursive>
 8000916:	89ab      	ldrh	r3, [r5, #12]
 8000918:	071b      	lsls	r3, r3, #28
 800091a:	d501      	bpl.n	8000920 <_vfiprintf_r+0x3c>
 800091c:	692b      	ldr	r3, [r5, #16]
 800091e:	b9eb      	cbnz	r3, 800095c <_vfiprintf_r+0x78>
 8000920:	4629      	mov	r1, r5
 8000922:	4630      	mov	r0, r6
 8000924:	f000 fb5a 	bl	8000fdc <__swsetup_r>
 8000928:	b1c0      	cbz	r0, 800095c <_vfiprintf_r+0x78>
 800092a:	6e6b      	ldr	r3, [r5, #100]	; 0x64
 800092c:	07dc      	lsls	r4, r3, #31
 800092e:	d50e      	bpl.n	800094e <_vfiprintf_r+0x6a>
 8000930:	f04f 30ff 	mov.w	r0, #4294967295
 8000934:	b01d      	add	sp, #116	; 0x74
 8000936:	e8bd 8ff0 	ldmia.w	sp!, {r4, r5, r6, r7, r8, r9, sl, fp, pc}
 800093a:	4b7b      	ldr	r3, [pc, #492]	; (8000b28 <_vfiprintf_r+0x244>)
 800093c:	429d      	cmp	r5, r3
 800093e:	d101      	bne.n	8000944 <_vfiprintf_r+0x60>
 8000940:	68b5      	ldr	r5, [r6, #8]
 8000942:	e7df      	b.n	8000904 <_vfiprintf_r+0x20>
 8000944:	4b79      	ldr	r3, [pc, #484]	; (8000b2c <_vfiprintf_r+0x248>)
 8000946:	429d      	cmp	r5, r3
 8000948:	bf08      	it	eq
 800094a:	68f5      	ldreq	r5, [r6, #12]
 800094c:	e7da      	b.n	8000904 <_vfiprintf_r+0x20>
 800094e:	89ab      	ldrh	r3, [r5, #12]
 8000950:	0598      	lsls	r0, r3, #22
 8000952:	d4ed      	bmi.n	8000930 <_vfiprintf_r+0x4c>
 8000954:	6da8      	ldr	r0, [r5, #88]	; 0x58
 8000956:	f7ff ff40 	bl	80007da <__retarget_lock_release_recursive>
 800095a:	e7e9      	b.n	8000930 <_vfiprintf_r+0x4c>
 800095c:	2300      	movs	r3, #0
 800095e:	9309      	str	r3, [sp, #36]	; 0x24
 8000960:	2320      	movs	r3, #32
 8000962:	f88d 3029 	strb.w	r3, [sp, #41]	; 0x29
 8000966:	f8cd 800c 	str.w	r8, [sp, #12]
 800096a:	2330      	movs	r3, #48	; 0x30
 800096c:	f8df 81c0 	ldr.w	r8, [pc, #448]	; 8000b30 <_vfiprintf_r+0x24c>
 8000970:	f88d 302a 	strb.w	r3, [sp, #42]	; 0x2a
 8000974:	f04f 0901 	mov.w	r9, #1
 8000978:	4623      	mov	r3, r4
 800097a:	469a      	mov	sl, r3
 800097c:	f813 2b01 	ldrb.w	r2, [r3], #1
 8000980:	b10a      	cbz	r2, 8000986 <_vfiprintf_r+0xa2>
 8000982:	2a25      	cmp	r2, #37	; 0x25
 8000984:	d1f9      	bne.n	800097a <_vfiprintf_r+0x96>
 8000986:	ebba 0b04 	subs.w	fp, sl, r4
 800098a:	d00b      	beq.n	80009a4 <_vfiprintf_r+0xc0>
 800098c:	465b      	mov	r3, fp
 800098e:	4622      	mov	r2, r4
 8000990:	4629      	mov	r1, r5
 8000992:	4630      	mov	r0, r6
 8000994:	f7ff ff93 	bl	80008be <__sfputs_r>
 8000998:	3001      	adds	r0, #1
 800099a:	f000 80aa 	beq.w	8000af2 <_vfiprintf_r+0x20e>
 800099e:	9a09      	ldr	r2, [sp, #36]	; 0x24
 80009a0:	445a      	add	r2, fp
 80009a2:	9209      	str	r2, [sp, #36]	; 0x24
 80009a4:	f89a 3000 	ldrb.w	r3, [sl]
 80009a8:	2b00      	cmp	r3, #0
 80009aa:	f000 80a2 	beq.w	8000af2 <_vfiprintf_r+0x20e>
 80009ae:	2300      	movs	r3, #0
 80009b0:	f04f 32ff 	mov.w	r2, #4294967295
 80009b4:	e9cd 2305 	strd	r2, r3, [sp, #20]
 80009b8:	f10a 0a01 	add.w	sl, sl, #1
 80009bc:	9304      	str	r3, [sp, #16]
 80009be:	9307      	str	r3, [sp, #28]
 80009c0:	f88d 3053 	strb.w	r3, [sp, #83]	; 0x53
 80009c4:	931a      	str	r3, [sp, #104]	; 0x68
 80009c6:	4654      	mov	r4, sl
 80009c8:	2205      	movs	r2, #5
 80009ca:	f814 1b01 	ldrb.w	r1, [r4], #1
 80009ce:	4858      	ldr	r0, [pc, #352]	; (8000b30 <_vfiprintf_r+0x24c>)
 80009d0:	f7ff fc06 	bl	80001e0 <memchr>
 80009d4:	9a04      	ldr	r2, [sp, #16]
 80009d6:	b9d8      	cbnz	r0, 8000a10 <_vfiprintf_r+0x12c>
 80009d8:	06d1      	lsls	r1, r2, #27
 80009da:	bf44      	itt	mi
 80009dc:	2320      	movmi	r3, #32
 80009de:	f88d 3053 	strbmi.w	r3, [sp, #83]	; 0x53
 80009e2:	0713      	lsls	r3, r2, #28
 80009e4:	bf44      	itt	mi
 80009e6:	232b      	movmi	r3, #43	; 0x2b
 80009e8:	f88d 3053 	strbmi.w	r3, [sp, #83]	; 0x53
 80009ec:	f89a 3000 	ldrb.w	r3, [sl]
 80009f0:	2b2a      	cmp	r3, #42	; 0x2a
 80009f2:	d015      	beq.n	8000a20 <_vfiprintf_r+0x13c>
 80009f4:	9a07      	ldr	r2, [sp, #28]
 80009f6:	4654      	mov	r4, sl
 80009f8:	2000      	movs	r0, #0
 80009fa:	f04f 0c0a 	mov.w	ip, #10
 80009fe:	4621      	mov	r1, r4
 8000a00:	f811 3b01 	ldrb.w	r3, [r1], #1
 8000a04:	3b30      	subs	r3, #48	; 0x30
 8000a06:	2b09      	cmp	r3, #9
 8000a08:	d94e      	bls.n	8000aa8 <_vfiprintf_r+0x1c4>
 8000a0a:	b1b0      	cbz	r0, 8000a3a <_vfiprintf_r+0x156>
 8000a0c:	9207      	str	r2, [sp, #28]
 8000a0e:	e014      	b.n	8000a3a <_vfiprintf_r+0x156>
 8000a10:	eba0 0308 	sub.w	r3, r0, r8
 8000a14:	fa09 f303 	lsl.w	r3, r9, r3
 8000a18:	4313      	orrs	r3, r2
 8000a1a:	9304      	str	r3, [sp, #16]
 8000a1c:	46a2      	mov	sl, r4
 8000a1e:	e7d2      	b.n	80009c6 <_vfiprintf_r+0xe2>
 8000a20:	9b03      	ldr	r3, [sp, #12]
 8000a22:	1d19      	adds	r1, r3, #4
 8000a24:	681b      	ldr	r3, [r3, #0]
 8000a26:	9103      	str	r1, [sp, #12]
 8000a28:	2b00      	cmp	r3, #0
 8000a2a:	bfbb      	ittet	lt
 8000a2c:	425b      	neglt	r3, r3
 8000a2e:	f042 0202 	orrlt.w	r2, r2, #2
 8000a32:	9307      	strge	r3, [sp, #28]
 8000a34:	9307      	strlt	r3, [sp, #28]
 8000a36:	bfb8      	it	lt
 8000a38:	9204      	strlt	r2, [sp, #16]
 8000a3a:	7823      	ldrb	r3, [r4, #0]
 8000a3c:	2b2e      	cmp	r3, #46	; 0x2e
 8000a3e:	d10c      	bne.n	8000a5a <_vfiprintf_r+0x176>
 8000a40:	7863      	ldrb	r3, [r4, #1]
 8000a42:	2b2a      	cmp	r3, #42	; 0x2a
 8000a44:	d135      	bne.n	8000ab2 <_vfiprintf_r+0x1ce>
 8000a46:	9b03      	ldr	r3, [sp, #12]
 8000a48:	1d1a      	adds	r2, r3, #4
 8000a4a:	681b      	ldr	r3, [r3, #0]
 8000a4c:	9203      	str	r2, [sp, #12]
 8000a4e:	2b00      	cmp	r3, #0
 8000a50:	bfb8      	it	lt
 8000a52:	f04f 33ff 	movlt.w	r3, #4294967295
 8000a56:	3402      	adds	r4, #2
 8000a58:	9305      	str	r3, [sp, #20]
 8000a5a:	f8df a0e4 	ldr.w	sl, [pc, #228]	; 8000b40 <_vfiprintf_r+0x25c>
 8000a5e:	7821      	ldrb	r1, [r4, #0]
 8000a60:	2203      	movs	r2, #3
 8000a62:	4650      	mov	r0, sl
 8000a64:	f7ff fbbc 	bl	80001e0 <memchr>
 8000a68:	b140      	cbz	r0, 8000a7c <_vfiprintf_r+0x198>
 8000a6a:	2340      	movs	r3, #64	; 0x40
 8000a6c:	eba0 000a 	sub.w	r0, r0, sl
 8000a70:	fa03 f000 	lsl.w	r0, r3, r0
 8000a74:	9b04      	ldr	r3, [sp, #16]
 8000a76:	4303      	orrs	r3, r0
 8000a78:	3401      	adds	r4, #1
 8000a7a:	9304      	str	r3, [sp, #16]
 8000a7c:	f814 1b01 	ldrb.w	r1, [r4], #1
 8000a80:	482c      	ldr	r0, [pc, #176]	; (8000b34 <_vfiprintf_r+0x250>)
 8000a82:	f88d 1028 	strb.w	r1, [sp, #40]	; 0x28
 8000a86:	2206      	movs	r2, #6
 8000a88:	f7ff fbaa 	bl	80001e0 <memchr>
 8000a8c:	2800      	cmp	r0, #0
 8000a8e:	d03f      	beq.n	8000b10 <_vfiprintf_r+0x22c>
 8000a90:	4b29      	ldr	r3, [pc, #164]	; (8000b38 <_vfiprintf_r+0x254>)
 8000a92:	bb1b      	cbnz	r3, 8000adc <_vfiprintf_r+0x1f8>
 8000a94:	9b03      	ldr	r3, [sp, #12]
 8000a96:	3307      	adds	r3, #7
 8000a98:	f023 0307 	bic.w	r3, r3, #7
 8000a9c:	3308      	adds	r3, #8
 8000a9e:	9303      	str	r3, [sp, #12]
 8000aa0:	9b09      	ldr	r3, [sp, #36]	; 0x24
 8000aa2:	443b      	add	r3, r7
 8000aa4:	9309      	str	r3, [sp, #36]	; 0x24
 8000aa6:	e767      	b.n	8000978 <_vfiprintf_r+0x94>
 8000aa8:	fb0c 3202 	mla	r2, ip, r2, r3
 8000aac:	460c      	mov	r4, r1
 8000aae:	2001      	movs	r0, #1
 8000ab0:	e7a5      	b.n	80009fe <_vfiprintf_r+0x11a>
 8000ab2:	2300      	movs	r3, #0
 8000ab4:	3401      	adds	r4, #1
 8000ab6:	9305      	str	r3, [sp, #20]
 8000ab8:	4619      	mov	r1, r3
 8000aba:	f04f 0c0a 	mov.w	ip, #10
 8000abe:	4620      	mov	r0, r4
 8000ac0:	f810 2b01 	ldrb.w	r2, [r0], #1
 8000ac4:	3a30      	subs	r2, #48	; 0x30
 8000ac6:	2a09      	cmp	r2, #9
 8000ac8:	d903      	bls.n	8000ad2 <_vfiprintf_r+0x1ee>
 8000aca:	2b00      	cmp	r3, #0
 8000acc:	d0c5      	beq.n	8000a5a <_vfiprintf_r+0x176>
 8000ace:	9105      	str	r1, [sp, #20]
 8000ad0:	e7c3      	b.n	8000a5a <_vfiprintf_r+0x176>
 8000ad2:	fb0c 2101 	mla	r1, ip, r1, r2
 8000ad6:	4604      	mov	r4, r0
 8000ad8:	2301      	movs	r3, #1
 8000ada:	e7f0      	b.n	8000abe <_vfiprintf_r+0x1da>
 8000adc:	ab03      	add	r3, sp, #12
 8000ade:	9300      	str	r3, [sp, #0]
 8000ae0:	462a      	mov	r2, r5
 8000ae2:	4b16      	ldr	r3, [pc, #88]	; (8000b3c <_vfiprintf_r+0x258>)
 8000ae4:	a904      	add	r1, sp, #16
 8000ae6:	4630      	mov	r0, r6
 8000ae8:	f3af 8000 	nop.w
 8000aec:	4607      	mov	r7, r0
 8000aee:	1c78      	adds	r0, r7, #1
 8000af0:	d1d6      	bne.n	8000aa0 <_vfiprintf_r+0x1bc>
 8000af2:	6e6b      	ldr	r3, [r5, #100]	; 0x64
 8000af4:	07d9      	lsls	r1, r3, #31
 8000af6:	d405      	bmi.n	8000b04 <_vfiprintf_r+0x220>
 8000af8:	89ab      	ldrh	r3, [r5, #12]
 8000afa:	059a      	lsls	r2, r3, #22
 8000afc:	d402      	bmi.n	8000b04 <_vfiprintf_r+0x220>
 8000afe:	6da8      	ldr	r0, [r5, #88]	; 0x58
 8000b00:	f7ff fe6b 	bl	80007da <__retarget_lock_release_recursive>
 8000b04:	89ab      	ldrh	r3, [r5, #12]
 8000b06:	065b      	lsls	r3, r3, #25
 8000b08:	f53f af12 	bmi.w	8000930 <_vfiprintf_r+0x4c>
 8000b0c:	9809      	ldr	r0, [sp, #36]	; 0x24
 8000b0e:	e711      	b.n	8000934 <_vfiprintf_r+0x50>
 8000b10:	ab03      	add	r3, sp, #12
 8000b12:	9300      	str	r3, [sp, #0]
 8000b14:	462a      	mov	r2, r5
 8000b16:	4b09      	ldr	r3, [pc, #36]	; (8000b3c <_vfiprintf_r+0x258>)
 8000b18:	a904      	add	r1, sp, #16
 8000b1a:	4630      	mov	r0, r6
 8000b1c:	f000 f880 	bl	8000c20 <_printf_i>
 8000b20:	e7e4      	b.n	8000aec <_vfiprintf_r+0x208>
 8000b22:	bf00      	nop
 8000b24:	080014b0 	.word	0x080014b0
 8000b28:	080014d0 	.word	0x080014d0
 8000b2c:	08001490 	.word	0x08001490
 8000b30:	080014f0 	.word	0x080014f0
 8000b34:	080014fa 	.word	0x080014fa
 8000b38:	00000000 	.word	0x00000000
 8000b3c:	080008bf 	.word	0x080008bf
 8000b40:	080014f6 	.word	0x080014f6

08000b44 <_printf_common>:
 8000b44:	e92d 47f0 	stmdb	sp!, {r4, r5, r6, r7, r8, r9, sl, lr}
 8000b48:	4616      	mov	r6, r2
 8000b4a:	4699      	mov	r9, r3
 8000b4c:	688a      	ldr	r2, [r1, #8]
 8000b4e:	690b      	ldr	r3, [r1, #16]
 8000b50:	f8dd 8020 	ldr.w	r8, [sp, #32]
 8000b54:	4293      	cmp	r3, r2
 8000b56:	bfb8      	it	lt
 8000b58:	4613      	movlt	r3, r2
 8000b5a:	6033      	str	r3, [r6, #0]
 8000b5c:	f891 2043 	ldrb.w	r2, [r1, #67]	; 0x43
 8000b60:	4607      	mov	r7, r0
 8000b62:	460c      	mov	r4, r1
 8000b64:	b10a      	cbz	r2, 8000b6a <_printf_common+0x26>
 8000b66:	3301      	adds	r3, #1
 8000b68:	6033      	str	r3, [r6, #0]
 8000b6a:	6823      	ldr	r3, [r4, #0]
 8000b6c:	0699      	lsls	r1, r3, #26
 8000b6e:	bf42      	ittt	mi
 8000b70:	6833      	ldrmi	r3, [r6, #0]
 8000b72:	3302      	addmi	r3, #2
 8000b74:	6033      	strmi	r3, [r6, #0]
 8000b76:	6825      	ldr	r5, [r4, #0]
 8000b78:	f015 0506 	ands.w	r5, r5, #6
 8000b7c:	d106      	bne.n	8000b8c <_printf_common+0x48>
 8000b7e:	f104 0a19 	add.w	sl, r4, #25
 8000b82:	68e3      	ldr	r3, [r4, #12]
 8000b84:	6832      	ldr	r2, [r6, #0]
 8000b86:	1a9b      	subs	r3, r3, r2
 8000b88:	42ab      	cmp	r3, r5
 8000b8a:	dc26      	bgt.n	8000bda <_printf_common+0x96>
 8000b8c:	f894 2043 	ldrb.w	r2, [r4, #67]	; 0x43
 8000b90:	1e13      	subs	r3, r2, #0
 8000b92:	6822      	ldr	r2, [r4, #0]
 8000b94:	bf18      	it	ne
 8000b96:	2301      	movne	r3, #1
 8000b98:	0692      	lsls	r2, r2, #26
 8000b9a:	d42b      	bmi.n	8000bf4 <_printf_common+0xb0>
 8000b9c:	f104 0243 	add.w	r2, r4, #67	; 0x43
 8000ba0:	4649      	mov	r1, r9
 8000ba2:	4638      	mov	r0, r7
 8000ba4:	47c0      	blx	r8
 8000ba6:	3001      	adds	r0, #1
 8000ba8:	d01e      	beq.n	8000be8 <_printf_common+0xa4>
 8000baa:	6823      	ldr	r3, [r4, #0]
 8000bac:	68e5      	ldr	r5, [r4, #12]
 8000bae:	6832      	ldr	r2, [r6, #0]
 8000bb0:	f003 0306 	and.w	r3, r3, #6
 8000bb4:	2b04      	cmp	r3, #4
 8000bb6:	bf08      	it	eq
 8000bb8:	1aad      	subeq	r5, r5, r2
 8000bba:	68a3      	ldr	r3, [r4, #8]
 8000bbc:	6922      	ldr	r2, [r4, #16]
 8000bbe:	bf0c      	ite	eq
 8000bc0:	ea25 75e5 	biceq.w	r5, r5, r5, asr #31
 8000bc4:	2500      	movne	r5, #0
 8000bc6:	4293      	cmp	r3, r2
 8000bc8:	bfc4      	itt	gt
 8000bca:	1a9b      	subgt	r3, r3, r2
 8000bcc:	18ed      	addgt	r5, r5, r3
 8000bce:	2600      	movs	r6, #0
 8000bd0:	341a      	adds	r4, #26
 8000bd2:	42b5      	cmp	r5, r6
 8000bd4:	d11a      	bne.n	8000c0c <_printf_common+0xc8>
 8000bd6:	2000      	movs	r0, #0
 8000bd8:	e008      	b.n	8000bec <_printf_common+0xa8>
 8000bda:	2301      	movs	r3, #1
 8000bdc:	4652      	mov	r2, sl
 8000bde:	4649      	mov	r1, r9
 8000be0:	4638      	mov	r0, r7
 8000be2:	47c0      	blx	r8
 8000be4:	3001      	adds	r0, #1
 8000be6:	d103      	bne.n	8000bf0 <_printf_common+0xac>
 8000be8:	f04f 30ff 	mov.w	r0, #4294967295
 8000bec:	e8bd 87f0 	ldmia.w	sp!, {r4, r5, r6, r7, r8, r9, sl, pc}
 8000bf0:	3501      	adds	r5, #1
 8000bf2:	e7c6      	b.n	8000b82 <_printf_common+0x3e>
 8000bf4:	18e1      	adds	r1, r4, r3
 8000bf6:	1c5a      	adds	r2, r3, #1
 8000bf8:	2030      	movs	r0, #48	; 0x30
 8000bfa:	f881 0043 	strb.w	r0, [r1, #67]	; 0x43
 8000bfe:	4422      	add	r2, r4
 8000c00:	f894 1045 	ldrb.w	r1, [r4, #69]	; 0x45
 8000c04:	f882 1043 	strb.w	r1, [r2, #67]	; 0x43
 8000c08:	3302      	adds	r3, #2
 8000c0a:	e7c7      	b.n	8000b9c <_printf_common+0x58>
 8000c0c:	2301      	movs	r3, #1
 8000c0e:	4622      	mov	r2, r4
 8000c10:	4649      	mov	r1, r9
 8000c12:	4638      	mov	r0, r7
 8000c14:	47c0      	blx	r8
 8000c16:	3001      	adds	r0, #1
 8000c18:	d0e6      	beq.n	8000be8 <_printf_common+0xa4>
 8000c1a:	3601      	adds	r6, #1
 8000c1c:	e7d9      	b.n	8000bd2 <_printf_common+0x8e>
	...

08000c20 <_printf_i>:
 8000c20:	e92d 47ff 	stmdb	sp!, {r0, r1, r2, r3, r4, r5, r6, r7, r8, r9, sl, lr}
 8000c24:	460c      	mov	r4, r1
 8000c26:	4691      	mov	r9, r2
 8000c28:	7e27      	ldrb	r7, [r4, #24]
 8000c2a:	990c      	ldr	r1, [sp, #48]	; 0x30
 8000c2c:	2f78      	cmp	r7, #120	; 0x78
 8000c2e:	4680      	mov	r8, r0
 8000c30:	469a      	mov	sl, r3
 8000c32:	f104 0243 	add.w	r2, r4, #67	; 0x43
 8000c36:	d807      	bhi.n	8000c48 <_printf_i+0x28>
 8000c38:	2f62      	cmp	r7, #98	; 0x62
 8000c3a:	d80a      	bhi.n	8000c52 <_printf_i+0x32>
 8000c3c:	2f00      	cmp	r7, #0
 8000c3e:	f000 80d8 	beq.w	8000df2 <_printf_i+0x1d2>
 8000c42:	2f58      	cmp	r7, #88	; 0x58
 8000c44:	f000 80a3 	beq.w	8000d8e <_printf_i+0x16e>
 8000c48:	f104 0642 	add.w	r6, r4, #66	; 0x42
 8000c4c:	f884 7042 	strb.w	r7, [r4, #66]	; 0x42
 8000c50:	e03a      	b.n	8000cc8 <_printf_i+0xa8>
 8000c52:	f1a7 0363 	sub.w	r3, r7, #99	; 0x63
 8000c56:	2b15      	cmp	r3, #21
 8000c58:	d8f6      	bhi.n	8000c48 <_printf_i+0x28>
 8000c5a:	a001      	add	r0, pc, #4	; (adr r0, 8000c60 <_printf_i+0x40>)
 8000c5c:	f850 f023 	ldr.w	pc, [r0, r3, lsl #2]
 8000c60:	08000cb9 	.word	0x08000cb9
 8000c64:	08000ccd 	.word	0x08000ccd
 8000c68:	08000c49 	.word	0x08000c49
 8000c6c:	08000c49 	.word	0x08000c49
 8000c70:	08000c49 	.word	0x08000c49
 8000c74:	08000c49 	.word	0x08000c49
 8000c78:	08000ccd 	.word	0x08000ccd
 8000c7c:	08000c49 	.word	0x08000c49
 8000c80:	08000c49 	.word	0x08000c49
 8000c84:	08000c49 	.word	0x08000c49
 8000c88:	08000c49 	.word	0x08000c49
 8000c8c:	08000dd9 	.word	0x08000dd9
 8000c90:	08000cfd 	.word	0x08000cfd
 8000c94:	08000dbb 	.word	0x08000dbb
 8000c98:	08000c49 	.word	0x08000c49
 8000c9c:	08000c49 	.word	0x08000c49
 8000ca0:	08000dfb 	.word	0x08000dfb
 8000ca4:	08000c49 	.word	0x08000c49
 8000ca8:	08000cfd 	.word	0x08000cfd
 8000cac:	08000c49 	.word	0x08000c49
 8000cb0:	08000c49 	.word	0x08000c49
 8000cb4:	08000dc3 	.word	0x08000dc3
 8000cb8:	680b      	ldr	r3, [r1, #0]
 8000cba:	1d1a      	adds	r2, r3, #4
 8000cbc:	681b      	ldr	r3, [r3, #0]
 8000cbe:	600a      	str	r2, [r1, #0]
 8000cc0:	f104 0642 	add.w	r6, r4, #66	; 0x42
 8000cc4:	f884 3042 	strb.w	r3, [r4, #66]	; 0x42
 8000cc8:	2301      	movs	r3, #1
 8000cca:	e0a3      	b.n	8000e14 <_printf_i+0x1f4>
 8000ccc:	6825      	ldr	r5, [r4, #0]
 8000cce:	6808      	ldr	r0, [r1, #0]
 8000cd0:	062e      	lsls	r6, r5, #24
 8000cd2:	f100 0304 	add.w	r3, r0, #4
 8000cd6:	d50a      	bpl.n	8000cee <_printf_i+0xce>
 8000cd8:	6805      	ldr	r5, [r0, #0]
 8000cda:	600b      	str	r3, [r1, #0]
 8000cdc:	2d00      	cmp	r5, #0
 8000cde:	da03      	bge.n	8000ce8 <_printf_i+0xc8>
 8000ce0:	232d      	movs	r3, #45	; 0x2d
 8000ce2:	426d      	negs	r5, r5
 8000ce4:	f884 3043 	strb.w	r3, [r4, #67]	; 0x43
 8000ce8:	485e      	ldr	r0, [pc, #376]	; (8000e64 <_printf_i+0x244>)
 8000cea:	230a      	movs	r3, #10
 8000cec:	e019      	b.n	8000d22 <_printf_i+0x102>
 8000cee:	f015 0f40 	tst.w	r5, #64	; 0x40
 8000cf2:	6805      	ldr	r5, [r0, #0]
 8000cf4:	600b      	str	r3, [r1, #0]
 8000cf6:	bf18      	it	ne
 8000cf8:	b22d      	sxthne	r5, r5
 8000cfa:	e7ef      	b.n	8000cdc <_printf_i+0xbc>
 8000cfc:	680b      	ldr	r3, [r1, #0]
 8000cfe:	6825      	ldr	r5, [r4, #0]
 8000d00:	1d18      	adds	r0, r3, #4
 8000d02:	6008      	str	r0, [r1, #0]
 8000d04:	0628      	lsls	r0, r5, #24
 8000d06:	d501      	bpl.n	8000d0c <_printf_i+0xec>
 8000d08:	681d      	ldr	r5, [r3, #0]
 8000d0a:	e002      	b.n	8000d12 <_printf_i+0xf2>
 8000d0c:	0669      	lsls	r1, r5, #25
 8000d0e:	d5fb      	bpl.n	8000d08 <_printf_i+0xe8>
 8000d10:	881d      	ldrh	r5, [r3, #0]
 8000d12:	4854      	ldr	r0, [pc, #336]	; (8000e64 <_printf_i+0x244>)
 8000d14:	2f6f      	cmp	r7, #111	; 0x6f
 8000d16:	bf0c      	ite	eq
 8000d18:	2308      	moveq	r3, #8
 8000d1a:	230a      	movne	r3, #10
 8000d1c:	2100      	movs	r1, #0
 8000d1e:	f884 1043 	strb.w	r1, [r4, #67]	; 0x43
 8000d22:	6866      	ldr	r6, [r4, #4]
 8000d24:	60a6      	str	r6, [r4, #8]
 8000d26:	2e00      	cmp	r6, #0
 8000d28:	bfa2      	ittt	ge
 8000d2a:	6821      	ldrge	r1, [r4, #0]
 8000d2c:	f021 0104 	bicge.w	r1, r1, #4
 8000d30:	6021      	strge	r1, [r4, #0]
 8000d32:	b90d      	cbnz	r5, 8000d38 <_printf_i+0x118>
 8000d34:	2e00      	cmp	r6, #0
 8000d36:	d04d      	beq.n	8000dd4 <_printf_i+0x1b4>
 8000d38:	4616      	mov	r6, r2
 8000d3a:	fbb5 f1f3 	udiv	r1, r5, r3
 8000d3e:	fb03 5711 	mls	r7, r3, r1, r5
 8000d42:	5dc7      	ldrb	r7, [r0, r7]
 8000d44:	f806 7d01 	strb.w	r7, [r6, #-1]!
 8000d48:	462f      	mov	r7, r5
 8000d4a:	42bb      	cmp	r3, r7
 8000d4c:	460d      	mov	r5, r1
 8000d4e:	d9f4      	bls.n	8000d3a <_printf_i+0x11a>
 8000d50:	2b08      	cmp	r3, #8
 8000d52:	d10b      	bne.n	8000d6c <_printf_i+0x14c>
 8000d54:	6823      	ldr	r3, [r4, #0]
 8000d56:	07df      	lsls	r7, r3, #31
 8000d58:	d508      	bpl.n	8000d6c <_printf_i+0x14c>
 8000d5a:	6923      	ldr	r3, [r4, #16]
 8000d5c:	6861      	ldr	r1, [r4, #4]
 8000d5e:	4299      	cmp	r1, r3
 8000d60:	bfde      	ittt	le
 8000d62:	2330      	movle	r3, #48	; 0x30
 8000d64:	f806 3c01 	strble.w	r3, [r6, #-1]
 8000d68:	f106 36ff 	addle.w	r6, r6, #4294967295
 8000d6c:	1b92      	subs	r2, r2, r6
 8000d6e:	6122      	str	r2, [r4, #16]
 8000d70:	f8cd a000 	str.w	sl, [sp]
 8000d74:	464b      	mov	r3, r9
 8000d76:	aa03      	add	r2, sp, #12
 8000d78:	4621      	mov	r1, r4
 8000d7a:	4640      	mov	r0, r8
 8000d7c:	f7ff fee2 	bl	8000b44 <_printf_common>
 8000d80:	3001      	adds	r0, #1
 8000d82:	d14c      	bne.n	8000e1e <_printf_i+0x1fe>
 8000d84:	f04f 30ff 	mov.w	r0, #4294967295
 8000d88:	b004      	add	sp, #16
 8000d8a:	e8bd 87f0 	ldmia.w	sp!, {r4, r5, r6, r7, r8, r9, sl, pc}
 8000d8e:	4835      	ldr	r0, [pc, #212]	; (8000e64 <_printf_i+0x244>)
 8000d90:	f884 7045 	strb.w	r7, [r4, #69]	; 0x45
 8000d94:	6823      	ldr	r3, [r4, #0]
 8000d96:	680e      	ldr	r6, [r1, #0]
 8000d98:	061f      	lsls	r7, r3, #24
 8000d9a:	f856 5b04 	ldr.w	r5, [r6], #4
 8000d9e:	600e      	str	r6, [r1, #0]
 8000da0:	d514      	bpl.n	8000dcc <_printf_i+0x1ac>
 8000da2:	07d9      	lsls	r1, r3, #31
 8000da4:	bf44      	itt	mi
 8000da6:	f043 0320 	orrmi.w	r3, r3, #32
 8000daa:	6023      	strmi	r3, [r4, #0]
 8000dac:	b91d      	cbnz	r5, 8000db6 <_printf_i+0x196>
 8000dae:	6823      	ldr	r3, [r4, #0]
 8000db0:	f023 0320 	bic.w	r3, r3, #32
 8000db4:	6023      	str	r3, [r4, #0]
 8000db6:	2310      	movs	r3, #16
 8000db8:	e7b0      	b.n	8000d1c <_printf_i+0xfc>
 8000dba:	6823      	ldr	r3, [r4, #0]
 8000dbc:	f043 0320 	orr.w	r3, r3, #32
 8000dc0:	6023      	str	r3, [r4, #0]
 8000dc2:	2378      	movs	r3, #120	; 0x78
 8000dc4:	4828      	ldr	r0, [pc, #160]	; (8000e68 <_printf_i+0x248>)
 8000dc6:	f884 3045 	strb.w	r3, [r4, #69]	; 0x45
 8000dca:	e7e3      	b.n	8000d94 <_printf_i+0x174>
 8000dcc:	065e      	lsls	r6, r3, #25
 8000dce:	bf48      	it	mi
 8000dd0:	b2ad      	uxthmi	r5, r5
 8000dd2:	e7e6      	b.n	8000da2 <_printf_i+0x182>
 8000dd4:	4616      	mov	r6, r2
 8000dd6:	e7bb      	b.n	8000d50 <_printf_i+0x130>
 8000dd8:	680b      	ldr	r3, [r1, #0]
 8000dda:	6826      	ldr	r6, [r4, #0]
 8000ddc:	6960      	ldr	r0, [r4, #20]
 8000dde:	1d1d      	adds	r5, r3, #4
 8000de0:	600d      	str	r5, [r1, #0]
 8000de2:	0635      	lsls	r5, r6, #24
 8000de4:	681b      	ldr	r3, [r3, #0]
 8000de6:	d501      	bpl.n	8000dec <_printf_i+0x1cc>
 8000de8:	6018      	str	r0, [r3, #0]
 8000dea:	e002      	b.n	8000df2 <_printf_i+0x1d2>
 8000dec:	0671      	lsls	r1, r6, #25
 8000dee:	d5fb      	bpl.n	8000de8 <_printf_i+0x1c8>
 8000df0:	8018      	strh	r0, [r3, #0]
 8000df2:	2300      	movs	r3, #0
 8000df4:	6123      	str	r3, [r4, #16]
 8000df6:	4616      	mov	r6, r2
 8000df8:	e7ba      	b.n	8000d70 <_printf_i+0x150>
 8000dfa:	680b      	ldr	r3, [r1, #0]
 8000dfc:	1d1a      	adds	r2, r3, #4
 8000dfe:	600a      	str	r2, [r1, #0]
 8000e00:	681e      	ldr	r6, [r3, #0]
 8000e02:	6862      	ldr	r2, [r4, #4]
 8000e04:	2100      	movs	r1, #0
 8000e06:	4630      	mov	r0, r6
 8000e08:	f7ff f9ea 	bl	80001e0 <memchr>
 8000e0c:	b108      	cbz	r0, 8000e12 <_printf_i+0x1f2>
 8000e0e:	1b80      	subs	r0, r0, r6
 8000e10:	6060      	str	r0, [r4, #4]
 8000e12:	6863      	ldr	r3, [r4, #4]
 8000e14:	6123      	str	r3, [r4, #16]
 8000e16:	2300      	movs	r3, #0
 8000e18:	f884 3043 	strb.w	r3, [r4, #67]	; 0x43
 8000e1c:	e7a8      	b.n	8000d70 <_printf_i+0x150>
 8000e1e:	6923      	ldr	r3, [r4, #16]
 8000e20:	4632      	mov	r2, r6
 8000e22:	4649      	mov	r1, r9
 8000e24:	4640      	mov	r0, r8
 8000e26:	47d0      	blx	sl
 8000e28:	3001      	adds	r0, #1
 8000e2a:	d0ab      	beq.n	8000d84 <_printf_i+0x164>
 8000e2c:	6823      	ldr	r3, [r4, #0]
 8000e2e:	079b      	lsls	r3, r3, #30
 8000e30:	d413      	bmi.n	8000e5a <_printf_i+0x23a>
 8000e32:	68e0      	ldr	r0, [r4, #12]
 8000e34:	9b03      	ldr	r3, [sp, #12]
 8000e36:	4298      	cmp	r0, r3
 8000e38:	bfb8      	it	lt
 8000e3a:	4618      	movlt	r0, r3
 8000e3c:	e7a4      	b.n	8000d88 <_printf_i+0x168>
 8000e3e:	2301      	movs	r3, #1
 8000e40:	4632      	mov	r2, r6
 8000e42:	4649      	mov	r1, r9
 8000e44:	4640      	mov	r0, r8
 8000e46:	47d0      	blx	sl
 8000e48:	3001      	adds	r0, #1
 8000e4a:	d09b      	beq.n	8000d84 <_printf_i+0x164>
 8000e4c:	3501      	adds	r5, #1
 8000e4e:	68e3      	ldr	r3, [r4, #12]
 8000e50:	9903      	ldr	r1, [sp, #12]
 8000e52:	1a5b      	subs	r3, r3, r1
 8000e54:	42ab      	cmp	r3, r5
 8000e56:	dcf2      	bgt.n	8000e3e <_printf_i+0x21e>
 8000e58:	e7eb      	b.n	8000e32 <_printf_i+0x212>
 8000e5a:	2500      	movs	r5, #0
 8000e5c:	f104 0619 	add.w	r6, r4, #25
 8000e60:	e7f5      	b.n	8000e4e <_printf_i+0x22e>
 8000e62:	bf00      	nop
 8000e64:	08001501 	.word	0x08001501
 8000e68:	08001512 	.word	0x08001512

08000e6c <_sbrk_r>:
 8000e6c:	b538      	push	{r3, r4, r5, lr}
 8000e6e:	4d06      	ldr	r5, [pc, #24]	; (8000e88 <_sbrk_r+0x1c>)
 8000e70:	2300      	movs	r3, #0
 8000e72:	4604      	mov	r4, r0
 8000e74:	4608      	mov	r0, r1
 8000e76:	602b      	str	r3, [r5, #0]
 8000e78:	f7ff fa7a 	bl	8000370 <_sbrk>
 8000e7c:	1c43      	adds	r3, r0, #1
 8000e7e:	d102      	bne.n	8000e86 <_sbrk_r+0x1a>
 8000e80:	682b      	ldr	r3, [r5, #0]
 8000e82:	b103      	cbz	r3, 8000e86 <_sbrk_r+0x1a>
 8000e84:	6023      	str	r3, [r4, #0]
 8000e86:	bd38      	pop	{r3, r4, r5, pc}
 8000e88:	20000098 	.word	0x20000098

08000e8c <__sread>:
 8000e8c:	b510      	push	{r4, lr}
 8000e8e:	460c      	mov	r4, r1
 8000e90:	f9b1 100e 	ldrsh.w	r1, [r1, #14]
 8000e94:	f000 fab4 	bl	8001400 <_read_r>
 8000e98:	2800      	cmp	r0, #0
 8000e9a:	bfab      	itete	ge
 8000e9c:	6d63      	ldrge	r3, [r4, #84]	; 0x54
 8000e9e:	89a3      	ldrhlt	r3, [r4, #12]
 8000ea0:	181b      	addge	r3, r3, r0
 8000ea2:	f423 5380 	biclt.w	r3, r3, #4096	; 0x1000
 8000ea6:	bfac      	ite	ge
 8000ea8:	6563      	strge	r3, [r4, #84]	; 0x54
 8000eaa:	81a3      	strhlt	r3, [r4, #12]
 8000eac:	bd10      	pop	{r4, pc}

08000eae <__swrite>:
 8000eae:	e92d 41f0 	stmdb	sp!, {r4, r5, r6, r7, r8, lr}
 8000eb2:	461f      	mov	r7, r3
 8000eb4:	898b      	ldrh	r3, [r1, #12]
 8000eb6:	05db      	lsls	r3, r3, #23
 8000eb8:	4605      	mov	r5, r0
 8000eba:	460c      	mov	r4, r1
 8000ebc:	4616      	mov	r6, r2
 8000ebe:	d505      	bpl.n	8000ecc <__swrite+0x1e>
 8000ec0:	f9b1 100e 	ldrsh.w	r1, [r1, #14]
 8000ec4:	2302      	movs	r3, #2
 8000ec6:	2200      	movs	r2, #0
 8000ec8:	f000 f9c8 	bl	800125c <_lseek_r>
 8000ecc:	89a3      	ldrh	r3, [r4, #12]
 8000ece:	f9b4 100e 	ldrsh.w	r1, [r4, #14]
 8000ed2:	f423 5380 	bic.w	r3, r3, #4096	; 0x1000
 8000ed6:	81a3      	strh	r3, [r4, #12]
 8000ed8:	4632      	mov	r2, r6
 8000eda:	463b      	mov	r3, r7
 8000edc:	4628      	mov	r0, r5
 8000ede:	e8bd 41f0 	ldmia.w	sp!, {r4, r5, r6, r7, r8, lr}
 8000ee2:	f000 b869 	b.w	8000fb8 <_write_r>

08000ee6 <__sseek>:
 8000ee6:	b510      	push	{r4, lr}
 8000ee8:	460c      	mov	r4, r1
 8000eea:	f9b1 100e 	ldrsh.w	r1, [r1, #14]
 8000eee:	f000 f9b5 	bl	800125c <_lseek_r>
 8000ef2:	1c43      	adds	r3, r0, #1
 8000ef4:	89a3      	ldrh	r3, [r4, #12]
 8000ef6:	bf15      	itete	ne
 8000ef8:	6560      	strne	r0, [r4, #84]	; 0x54
 8000efa:	f423 5380 	biceq.w	r3, r3, #4096	; 0x1000
 8000efe:	f443 5380 	orrne.w	r3, r3, #4096	; 0x1000
 8000f02:	81a3      	strheq	r3, [r4, #12]
 8000f04:	bf18      	it	ne
 8000f06:	81a3      	strhne	r3, [r4, #12]
 8000f08:	bd10      	pop	{r4, pc}

08000f0a <__sclose>:
 8000f0a:	f9b1 100e 	ldrsh.w	r1, [r1, #14]
 8000f0e:	f000 b8d3 	b.w	80010b8 <_close_r>
	...

08000f14 <__swbuf_r>:
 8000f14:	b5f8      	push	{r3, r4, r5, r6, r7, lr}
 8000f16:	460e      	mov	r6, r1
 8000f18:	4614      	mov	r4, r2
 8000f1a:	4605      	mov	r5, r0
 8000f1c:	b118      	cbz	r0, 8000f26 <__swbuf_r+0x12>
 8000f1e:	6983      	ldr	r3, [r0, #24]
 8000f20:	b90b      	cbnz	r3, 8000f26 <__swbuf_r+0x12>
 8000f22:	f7ff fbbb 	bl	800069c <__sinit>
 8000f26:	4b21      	ldr	r3, [pc, #132]	; (8000fac <__swbuf_r+0x98>)
 8000f28:	429c      	cmp	r4, r3
 8000f2a:	d12b      	bne.n	8000f84 <__swbuf_r+0x70>
 8000f2c:	686c      	ldr	r4, [r5, #4]
 8000f2e:	69a3      	ldr	r3, [r4, #24]
 8000f30:	60a3      	str	r3, [r4, #8]
 8000f32:	89a3      	ldrh	r3, [r4, #12]
 8000f34:	071a      	lsls	r2, r3, #28
 8000f36:	d52f      	bpl.n	8000f98 <__swbuf_r+0x84>
 8000f38:	6923      	ldr	r3, [r4, #16]
 8000f3a:	b36b      	cbz	r3, 8000f98 <__swbuf_r+0x84>
 8000f3c:	6923      	ldr	r3, [r4, #16]
 8000f3e:	6820      	ldr	r0, [r4, #0]
 8000f40:	1ac0      	subs	r0, r0, r3
 8000f42:	6963      	ldr	r3, [r4, #20]
 8000f44:	b2f6      	uxtb	r6, r6
 8000f46:	4283      	cmp	r3, r0
 8000f48:	4637      	mov	r7, r6
 8000f4a:	dc04      	bgt.n	8000f56 <__swbuf_r+0x42>
 8000f4c:	4621      	mov	r1, r4
 8000f4e:	4628      	mov	r0, r5
 8000f50:	f000 f948 	bl	80011e4 <_fflush_r>
 8000f54:	bb30      	cbnz	r0, 8000fa4 <__swbuf_r+0x90>
 8000f56:	68a3      	ldr	r3, [r4, #8]
 8000f58:	3b01      	subs	r3, #1
 8000f5a:	60a3      	str	r3, [r4, #8]
 8000f5c:	6823      	ldr	r3, [r4, #0]
 8000f5e:	1c5a      	adds	r2, r3, #1
 8000f60:	6022      	str	r2, [r4, #0]
 8000f62:	701e      	strb	r6, [r3, #0]
 8000f64:	6963      	ldr	r3, [r4, #20]
 8000f66:	3001      	adds	r0, #1
 8000f68:	4283      	cmp	r3, r0
 8000f6a:	d004      	beq.n	8000f76 <__swbuf_r+0x62>
 8000f6c:	89a3      	ldrh	r3, [r4, #12]
 8000f6e:	07db      	lsls	r3, r3, #31
 8000f70:	d506      	bpl.n	8000f80 <__swbuf_r+0x6c>
 8000f72:	2e0a      	cmp	r6, #10
 8000f74:	d104      	bne.n	8000f80 <__swbuf_r+0x6c>
 8000f76:	4621      	mov	r1, r4
 8000f78:	4628      	mov	r0, r5
 8000f7a:	f000 f933 	bl	80011e4 <_fflush_r>
 8000f7e:	b988      	cbnz	r0, 8000fa4 <__swbuf_r+0x90>
 8000f80:	4638      	mov	r0, r7
 8000f82:	bdf8      	pop	{r3, r4, r5, r6, r7, pc}
 8000f84:	4b0a      	ldr	r3, [pc, #40]	; (8000fb0 <__swbuf_r+0x9c>)
 8000f86:	429c      	cmp	r4, r3
 8000f88:	d101      	bne.n	8000f8e <__swbuf_r+0x7a>
 8000f8a:	68ac      	ldr	r4, [r5, #8]
 8000f8c:	e7cf      	b.n	8000f2e <__swbuf_r+0x1a>
 8000f8e:	4b09      	ldr	r3, [pc, #36]	; (8000fb4 <__swbuf_r+0xa0>)
 8000f90:	429c      	cmp	r4, r3
 8000f92:	bf08      	it	eq
 8000f94:	68ec      	ldreq	r4, [r5, #12]
 8000f96:	e7ca      	b.n	8000f2e <__swbuf_r+0x1a>
 8000f98:	4621      	mov	r1, r4
 8000f9a:	4628      	mov	r0, r5
 8000f9c:	f000 f81e 	bl	8000fdc <__swsetup_r>
 8000fa0:	2800      	cmp	r0, #0
 8000fa2:	d0cb      	beq.n	8000f3c <__swbuf_r+0x28>
 8000fa4:	f04f 37ff 	mov.w	r7, #4294967295
 8000fa8:	e7ea      	b.n	8000f80 <__swbuf_r+0x6c>
 8000faa:	bf00      	nop
 8000fac:	080014b0 	.word	0x080014b0
 8000fb0:	080014d0 	.word	0x080014d0
 8000fb4:	08001490 	.word	0x08001490

08000fb8 <_write_r>:
 8000fb8:	b538      	push	{r3, r4, r5, lr}
 8000fba:	4d07      	ldr	r5, [pc, #28]	; (8000fd8 <_write_r+0x20>)
 8000fbc:	4604      	mov	r4, r0
 8000fbe:	4608      	mov	r0, r1
 8000fc0:	4611      	mov	r1, r2
 8000fc2:	2200      	movs	r2, #0
 8000fc4:	602a      	str	r2, [r5, #0]
 8000fc6:	461a      	mov	r2, r3
 8000fc8:	f7ff f981 	bl	80002ce <_write>
 8000fcc:	1c43      	adds	r3, r0, #1
 8000fce:	d102      	bne.n	8000fd6 <_write_r+0x1e>
 8000fd0:	682b      	ldr	r3, [r5, #0]
 8000fd2:	b103      	cbz	r3, 8000fd6 <_write_r+0x1e>
 8000fd4:	6023      	str	r3, [r4, #0]
 8000fd6:	bd38      	pop	{r3, r4, r5, pc}
 8000fd8:	20000098 	.word	0x20000098

08000fdc <__swsetup_r>:
 8000fdc:	4b32      	ldr	r3, [pc, #200]	; (80010a8 <__swsetup_r+0xcc>)
 8000fde:	b570      	push	{r4, r5, r6, lr}
 8000fe0:	681d      	ldr	r5, [r3, #0]
 8000fe2:	4606      	mov	r6, r0
 8000fe4:	460c      	mov	r4, r1
 8000fe6:	b125      	cbz	r5, 8000ff2 <__swsetup_r+0x16>
 8000fe8:	69ab      	ldr	r3, [r5, #24]
 8000fea:	b913      	cbnz	r3, 8000ff2 <__swsetup_r+0x16>
 8000fec:	4628      	mov	r0, r5
 8000fee:	f7ff fb55 	bl	800069c <__sinit>
 8000ff2:	4b2e      	ldr	r3, [pc, #184]	; (80010ac <__swsetup_r+0xd0>)
 8000ff4:	429c      	cmp	r4, r3
 8000ff6:	d10f      	bne.n	8001018 <__swsetup_r+0x3c>
 8000ff8:	686c      	ldr	r4, [r5, #4]
 8000ffa:	89a3      	ldrh	r3, [r4, #12]
 8000ffc:	f9b4 200c 	ldrsh.w	r2, [r4, #12]
 8001000:	0719      	lsls	r1, r3, #28
 8001002:	d42c      	bmi.n	800105e <__swsetup_r+0x82>
 8001004:	06dd      	lsls	r5, r3, #27
 8001006:	d411      	bmi.n	800102c <__swsetup_r+0x50>
 8001008:	2309      	movs	r3, #9
 800100a:	6033      	str	r3, [r6, #0]
 800100c:	f042 0340 	orr.w	r3, r2, #64	; 0x40
 8001010:	81a3      	strh	r3, [r4, #12]
 8001012:	f04f 30ff 	mov.w	r0, #4294967295
 8001016:	e03e      	b.n	8001096 <__swsetup_r+0xba>
 8001018:	4b25      	ldr	r3, [pc, #148]	; (80010b0 <__swsetup_r+0xd4>)
 800101a:	429c      	cmp	r4, r3
 800101c:	d101      	bne.n	8001022 <__swsetup_r+0x46>
 800101e:	68ac      	ldr	r4, [r5, #8]
 8001020:	e7eb      	b.n	8000ffa <__swsetup_r+0x1e>
 8001022:	4b24      	ldr	r3, [pc, #144]	; (80010b4 <__swsetup_r+0xd8>)
 8001024:	429c      	cmp	r4, r3
 8001026:	bf08      	it	eq
 8001028:	68ec      	ldreq	r4, [r5, #12]
 800102a:	e7e6      	b.n	8000ffa <__swsetup_r+0x1e>
 800102c:	0758      	lsls	r0, r3, #29
 800102e:	d512      	bpl.n	8001056 <__swsetup_r+0x7a>
 8001030:	6b61      	ldr	r1, [r4, #52]	; 0x34
 8001032:	b141      	cbz	r1, 8001046 <__swsetup_r+0x6a>
 8001034:	f104 0344 	add.w	r3, r4, #68	; 0x44
 8001038:	4299      	cmp	r1, r3
 800103a:	d002      	beq.n	8001042 <__swsetup_r+0x66>
 800103c:	4630      	mov	r0, r6
 800103e:	f000 f98f 	bl	8001360 <_free_r>
 8001042:	2300      	movs	r3, #0
 8001044:	6363      	str	r3, [r4, #52]	; 0x34
 8001046:	89a3      	ldrh	r3, [r4, #12]
 8001048:	f023 0324 	bic.w	r3, r3, #36	; 0x24
 800104c:	81a3      	strh	r3, [r4, #12]
 800104e:	2300      	movs	r3, #0
 8001050:	6063      	str	r3, [r4, #4]
 8001052:	6923      	ldr	r3, [r4, #16]
 8001054:	6023      	str	r3, [r4, #0]
 8001056:	89a3      	ldrh	r3, [r4, #12]
 8001058:	f043 0308 	orr.w	r3, r3, #8
 800105c:	81a3      	strh	r3, [r4, #12]
 800105e:	6923      	ldr	r3, [r4, #16]
 8001060:	b94b      	cbnz	r3, 8001076 <__swsetup_r+0x9a>
 8001062:	89a3      	ldrh	r3, [r4, #12]
 8001064:	f403 7320 	and.w	r3, r3, #640	; 0x280
 8001068:	f5b3 7f00 	cmp.w	r3, #512	; 0x200
 800106c:	d003      	beq.n	8001076 <__swsetup_r+0x9a>
 800106e:	4621      	mov	r1, r4
 8001070:	4630      	mov	r0, r6
 8001072:	f000 f929 	bl	80012c8 <__smakebuf_r>
 8001076:	89a0      	ldrh	r0, [r4, #12]
 8001078:	f9b4 200c 	ldrsh.w	r2, [r4, #12]
 800107c:	f010 0301 	ands.w	r3, r0, #1
 8001080:	d00a      	beq.n	8001098 <__swsetup_r+0xbc>
 8001082:	2300      	movs	r3, #0
 8001084:	60a3      	str	r3, [r4, #8]
 8001086:	6963      	ldr	r3, [r4, #20]
 8001088:	425b      	negs	r3, r3
 800108a:	61a3      	str	r3, [r4, #24]
 800108c:	6923      	ldr	r3, [r4, #16]
 800108e:	b943      	cbnz	r3, 80010a2 <__swsetup_r+0xc6>
 8001090:	f010 0080 	ands.w	r0, r0, #128	; 0x80
 8001094:	d1ba      	bne.n	800100c <__swsetup_r+0x30>
 8001096:	bd70      	pop	{r4, r5, r6, pc}
 8001098:	0781      	lsls	r1, r0, #30
 800109a:	bf58      	it	pl
 800109c:	6963      	ldrpl	r3, [r4, #20]
 800109e:	60a3      	str	r3, [r4, #8]
 80010a0:	e7f4      	b.n	800108c <__swsetup_r+0xb0>
 80010a2:	2000      	movs	r0, #0
 80010a4:	e7f7      	b.n	8001096 <__swsetup_r+0xba>
 80010a6:	bf00      	nop
 80010a8:	20000000 	.word	0x20000000
 80010ac:	080014b0 	.word	0x080014b0
 80010b0:	080014d0 	.word	0x080014d0
 80010b4:	08001490 	.word	0x08001490

080010b8 <_close_r>:
 80010b8:	b538      	push	{r3, r4, r5, lr}
 80010ba:	4d06      	ldr	r5, [pc, #24]	; (80010d4 <_close_r+0x1c>)
 80010bc:	2300      	movs	r3, #0
 80010be:	4604      	mov	r4, r0
 80010c0:	4608      	mov	r0, r1
 80010c2:	602b      	str	r3, [r5, #0]
 80010c4:	f7ff f91f 	bl	8000306 <_close>
 80010c8:	1c43      	adds	r3, r0, #1
 80010ca:	d102      	bne.n	80010d2 <_close_r+0x1a>
 80010cc:	682b      	ldr	r3, [r5, #0]
 80010ce:	b103      	cbz	r3, 80010d2 <_close_r+0x1a>
 80010d0:	6023      	str	r3, [r4, #0]
 80010d2:	bd38      	pop	{r3, r4, r5, pc}
 80010d4:	20000098 	.word	0x20000098

080010d8 <__sflush_r>:
 80010d8:	898a      	ldrh	r2, [r1, #12]
 80010da:	e92d 41f0 	stmdb	sp!, {r4, r5, r6, r7, r8, lr}
 80010de:	4605      	mov	r5, r0
 80010e0:	0710      	lsls	r0, r2, #28
 80010e2:	460c      	mov	r4, r1
 80010e4:	d458      	bmi.n	8001198 <__sflush_r+0xc0>
 80010e6:	684b      	ldr	r3, [r1, #4]
 80010e8:	2b00      	cmp	r3, #0
 80010ea:	dc05      	bgt.n	80010f8 <__sflush_r+0x20>
 80010ec:	6c0b      	ldr	r3, [r1, #64]	; 0x40
 80010ee:	2b00      	cmp	r3, #0
 80010f0:	dc02      	bgt.n	80010f8 <__sflush_r+0x20>
 80010f2:	2000      	movs	r0, #0
 80010f4:	e8bd 81f0 	ldmia.w	sp!, {r4, r5, r6, r7, r8, pc}
 80010f8:	6ae6      	ldr	r6, [r4, #44]	; 0x2c
 80010fa:	2e00      	cmp	r6, #0
 80010fc:	d0f9      	beq.n	80010f2 <__sflush_r+0x1a>
 80010fe:	2300      	movs	r3, #0
 8001100:	f412 5280 	ands.w	r2, r2, #4096	; 0x1000
 8001104:	682f      	ldr	r7, [r5, #0]
 8001106:	602b      	str	r3, [r5, #0]
 8001108:	d032      	beq.n	8001170 <__sflush_r+0x98>
 800110a:	6d60      	ldr	r0, [r4, #84]	; 0x54
 800110c:	89a3      	ldrh	r3, [r4, #12]
 800110e:	075a      	lsls	r2, r3, #29
 8001110:	d505      	bpl.n	800111e <__sflush_r+0x46>
 8001112:	6863      	ldr	r3, [r4, #4]
 8001114:	1ac0      	subs	r0, r0, r3
 8001116:	6b63      	ldr	r3, [r4, #52]	; 0x34
 8001118:	b10b      	cbz	r3, 800111e <__sflush_r+0x46>
 800111a:	6c23      	ldr	r3, [r4, #64]	; 0x40
 800111c:	1ac0      	subs	r0, r0, r3
 800111e:	2300      	movs	r3, #0
 8001120:	4602      	mov	r2, r0
 8001122:	6ae6      	ldr	r6, [r4, #44]	; 0x2c
 8001124:	6a21      	ldr	r1, [r4, #32]
 8001126:	4628      	mov	r0, r5
 8001128:	47b0      	blx	r6
 800112a:	1c43      	adds	r3, r0, #1
 800112c:	89a3      	ldrh	r3, [r4, #12]
 800112e:	d106      	bne.n	800113e <__sflush_r+0x66>
 8001130:	6829      	ldr	r1, [r5, #0]
 8001132:	291d      	cmp	r1, #29
 8001134:	d82c      	bhi.n	8001190 <__sflush_r+0xb8>
 8001136:	4a2a      	ldr	r2, [pc, #168]	; (80011e0 <__sflush_r+0x108>)
 8001138:	40ca      	lsrs	r2, r1
 800113a:	07d6      	lsls	r6, r2, #31
 800113c:	d528      	bpl.n	8001190 <__sflush_r+0xb8>
 800113e:	2200      	movs	r2, #0
 8001140:	6062      	str	r2, [r4, #4]
 8001142:	04d9      	lsls	r1, r3, #19
 8001144:	6922      	ldr	r2, [r4, #16]
 8001146:	6022      	str	r2, [r4, #0]
 8001148:	d504      	bpl.n	8001154 <__sflush_r+0x7c>
 800114a:	1c42      	adds	r2, r0, #1
 800114c:	d101      	bne.n	8001152 <__sflush_r+0x7a>
 800114e:	682b      	ldr	r3, [r5, #0]
 8001150:	b903      	cbnz	r3, 8001154 <__sflush_r+0x7c>
 8001152:	6560      	str	r0, [r4, #84]	; 0x54
 8001154:	6b61      	ldr	r1, [r4, #52]	; 0x34
 8001156:	602f      	str	r7, [r5, #0]
 8001158:	2900      	cmp	r1, #0
 800115a:	d0ca      	beq.n	80010f2 <__sflush_r+0x1a>
 800115c:	f104 0344 	add.w	r3, r4, #68	; 0x44
 8001160:	4299      	cmp	r1, r3
 8001162:	d002      	beq.n	800116a <__sflush_r+0x92>
 8001164:	4628      	mov	r0, r5
 8001166:	f000 f8fb 	bl	8001360 <_free_r>
 800116a:	2000      	movs	r0, #0
 800116c:	6360      	str	r0, [r4, #52]	; 0x34
 800116e:	e7c1      	b.n	80010f4 <__sflush_r+0x1c>
 8001170:	6a21      	ldr	r1, [r4, #32]
 8001172:	2301      	movs	r3, #1
 8001174:	4628      	mov	r0, r5
 8001176:	47b0      	blx	r6
 8001178:	1c41      	adds	r1, r0, #1
 800117a:	d1c7      	bne.n	800110c <__sflush_r+0x34>
 800117c:	682b      	ldr	r3, [r5, #0]
 800117e:	2b00      	cmp	r3, #0
 8001180:	d0c4      	beq.n	800110c <__sflush_r+0x34>
 8001182:	2b1d      	cmp	r3, #29
 8001184:	d001      	beq.n	800118a <__sflush_r+0xb2>
 8001186:	2b16      	cmp	r3, #22
 8001188:	d101      	bne.n	800118e <__sflush_r+0xb6>
 800118a:	602f      	str	r7, [r5, #0]
 800118c:	e7b1      	b.n	80010f2 <__sflush_r+0x1a>
 800118e:	89a3      	ldrh	r3, [r4, #12]
 8001190:	f043 0340 	orr.w	r3, r3, #64	; 0x40
 8001194:	81a3      	strh	r3, [r4, #12]
 8001196:	e7ad      	b.n	80010f4 <__sflush_r+0x1c>
 8001198:	690f      	ldr	r7, [r1, #16]
 800119a:	2f00      	cmp	r7, #0
 800119c:	d0a9      	beq.n	80010f2 <__sflush_r+0x1a>
 800119e:	0793      	lsls	r3, r2, #30
 80011a0:	680e      	ldr	r6, [r1, #0]
 80011a2:	bf08      	it	eq
 80011a4:	694b      	ldreq	r3, [r1, #20]
 80011a6:	600f      	str	r7, [r1, #0]
 80011a8:	bf18      	it	ne
 80011aa:	2300      	movne	r3, #0
 80011ac:	eba6 0807 	sub.w	r8, r6, r7
 80011b0:	608b      	str	r3, [r1, #8]
 80011b2:	f1b8 0f00 	cmp.w	r8, #0
 80011b6:	dd9c      	ble.n	80010f2 <__sflush_r+0x1a>
 80011b8:	6a21      	ldr	r1, [r4, #32]
 80011ba:	6aa6      	ldr	r6, [r4, #40]	; 0x28
 80011bc:	4643      	mov	r3, r8
 80011be:	463a      	mov	r2, r7
 80011c0:	4628      	mov	r0, r5
 80011c2:	47b0      	blx	r6
 80011c4:	2800      	cmp	r0, #0
 80011c6:	dc06      	bgt.n	80011d6 <__sflush_r+0xfe>
 80011c8:	89a3      	ldrh	r3, [r4, #12]
 80011ca:	f043 0340 	orr.w	r3, r3, #64	; 0x40
 80011ce:	81a3      	strh	r3, [r4, #12]
 80011d0:	f04f 30ff 	mov.w	r0, #4294967295
 80011d4:	e78e      	b.n	80010f4 <__sflush_r+0x1c>
 80011d6:	4407      	add	r7, r0
 80011d8:	eba8 0800 	sub.w	r8, r8, r0
 80011dc:	e7e9      	b.n	80011b2 <__sflush_r+0xda>
 80011de:	bf00      	nop
 80011e0:	20400001 	.word	0x20400001

080011e4 <_fflush_r>:
 80011e4:	b538      	push	{r3, r4, r5, lr}
 80011e6:	690b      	ldr	r3, [r1, #16]
 80011e8:	4605      	mov	r5, r0
 80011ea:	460c      	mov	r4, r1
 80011ec:	b913      	cbnz	r3, 80011f4 <_fflush_r+0x10>
 80011ee:	2500      	movs	r5, #0
 80011f0:	4628      	mov	r0, r5
 80011f2:	bd38      	pop	{r3, r4, r5, pc}
 80011f4:	b118      	cbz	r0, 80011fe <_fflush_r+0x1a>
 80011f6:	6983      	ldr	r3, [r0, #24]
 80011f8:	b90b      	cbnz	r3, 80011fe <_fflush_r+0x1a>
 80011fa:	f7ff fa4f 	bl	800069c <__sinit>
 80011fe:	4b14      	ldr	r3, [pc, #80]	; (8001250 <_fflush_r+0x6c>)
 8001200:	429c      	cmp	r4, r3
 8001202:	d11b      	bne.n	800123c <_fflush_r+0x58>
 8001204:	686c      	ldr	r4, [r5, #4]
 8001206:	f9b4 300c 	ldrsh.w	r3, [r4, #12]
 800120a:	2b00      	cmp	r3, #0
 800120c:	d0ef      	beq.n	80011ee <_fflush_r+0xa>
 800120e:	6e62      	ldr	r2, [r4, #100]	; 0x64
 8001210:	07d0      	lsls	r0, r2, #31
 8001212:	d404      	bmi.n	800121e <_fflush_r+0x3a>
 8001214:	0599      	lsls	r1, r3, #22
 8001216:	d402      	bmi.n	800121e <_fflush_r+0x3a>
 8001218:	6da0      	ldr	r0, [r4, #88]	; 0x58
 800121a:	f7ff fadd 	bl	80007d8 <__retarget_lock_acquire_recursive>
 800121e:	4628      	mov	r0, r5
 8001220:	4621      	mov	r1, r4
 8001222:	f7ff ff59 	bl	80010d8 <__sflush_r>
 8001226:	6e63      	ldr	r3, [r4, #100]	; 0x64
 8001228:	07da      	lsls	r2, r3, #31
 800122a:	4605      	mov	r5, r0
 800122c:	d4e0      	bmi.n	80011f0 <_fflush_r+0xc>
 800122e:	89a3      	ldrh	r3, [r4, #12]
 8001230:	059b      	lsls	r3, r3, #22
 8001232:	d4dd      	bmi.n	80011f0 <_fflush_r+0xc>
 8001234:	6da0      	ldr	r0, [r4, #88]	; 0x58
 8001236:	f7ff fad0 	bl	80007da <__retarget_lock_release_recursive>
 800123a:	e7d9      	b.n	80011f0 <_fflush_r+0xc>
 800123c:	4b05      	ldr	r3, [pc, #20]	; (8001254 <_fflush_r+0x70>)
 800123e:	429c      	cmp	r4, r3
 8001240:	d101      	bne.n	8001246 <_fflush_r+0x62>
 8001242:	68ac      	ldr	r4, [r5, #8]
 8001244:	e7df      	b.n	8001206 <_fflush_r+0x22>
 8001246:	4b04      	ldr	r3, [pc, #16]	; (8001258 <_fflush_r+0x74>)
 8001248:	429c      	cmp	r4, r3
 800124a:	bf08      	it	eq
 800124c:	68ec      	ldreq	r4, [r5, #12]
 800124e:	e7da      	b.n	8001206 <_fflush_r+0x22>
 8001250:	080014b0 	.word	0x080014b0
 8001254:	080014d0 	.word	0x080014d0
 8001258:	08001490 	.word	0x08001490

0800125c <_lseek_r>:
 800125c:	b538      	push	{r3, r4, r5, lr}
 800125e:	4d07      	ldr	r5, [pc, #28]	; (800127c <_lseek_r+0x20>)
 8001260:	4604      	mov	r4, r0
 8001262:	4608      	mov	r0, r1
 8001264:	4611      	mov	r1, r2
 8001266:	2200      	movs	r2, #0
 8001268:	602a      	str	r2, [r5, #0]
 800126a:	461a      	mov	r2, r3
 800126c:	f7ff f872 	bl	8000354 <_lseek>
 8001270:	1c43      	adds	r3, r0, #1
 8001272:	d102      	bne.n	800127a <_lseek_r+0x1e>
 8001274:	682b      	ldr	r3, [r5, #0]
 8001276:	b103      	cbz	r3, 800127a <_lseek_r+0x1e>
 8001278:	6023      	str	r3, [r4, #0]
 800127a:	bd38      	pop	{r3, r4, r5, pc}
 800127c:	20000098 	.word	0x20000098

08001280 <__swhatbuf_r>:
 8001280:	b570      	push	{r4, r5, r6, lr}
 8001282:	460e      	mov	r6, r1
 8001284:	f9b1 100e 	ldrsh.w	r1, [r1, #14]
 8001288:	2900      	cmp	r1, #0
 800128a:	b096      	sub	sp, #88	; 0x58
 800128c:	4614      	mov	r4, r2
 800128e:	461d      	mov	r5, r3
 8001290:	da07      	bge.n	80012a2 <__swhatbuf_r+0x22>
 8001292:	2300      	movs	r3, #0
 8001294:	602b      	str	r3, [r5, #0]
 8001296:	89b3      	ldrh	r3, [r6, #12]
 8001298:	061a      	lsls	r2, r3, #24
 800129a:	d410      	bmi.n	80012be <__swhatbuf_r+0x3e>
 800129c:	f44f 6380 	mov.w	r3, #1024	; 0x400
 80012a0:	e00e      	b.n	80012c0 <__swhatbuf_r+0x40>
 80012a2:	466a      	mov	r2, sp
 80012a4:	f000 f8be 	bl	8001424 <_fstat_r>
 80012a8:	2800      	cmp	r0, #0
 80012aa:	dbf2      	blt.n	8001292 <__swhatbuf_r+0x12>
 80012ac:	9a01      	ldr	r2, [sp, #4]
 80012ae:	f402 4270 	and.w	r2, r2, #61440	; 0xf000
 80012b2:	f5a2 5300 	sub.w	r3, r2, #8192	; 0x2000
 80012b6:	425a      	negs	r2, r3
 80012b8:	415a      	adcs	r2, r3
 80012ba:	602a      	str	r2, [r5, #0]
 80012bc:	e7ee      	b.n	800129c <__swhatbuf_r+0x1c>
 80012be:	2340      	movs	r3, #64	; 0x40
 80012c0:	2000      	movs	r0, #0
 80012c2:	6023      	str	r3, [r4, #0]
 80012c4:	b016      	add	sp, #88	; 0x58
 80012c6:	bd70      	pop	{r4, r5, r6, pc}

080012c8 <__smakebuf_r>:
 80012c8:	898b      	ldrh	r3, [r1, #12]
 80012ca:	b573      	push	{r0, r1, r4, r5, r6, lr}
 80012cc:	079d      	lsls	r5, r3, #30
 80012ce:	4606      	mov	r6, r0
 80012d0:	460c      	mov	r4, r1
 80012d2:	d507      	bpl.n	80012e4 <__smakebuf_r+0x1c>
 80012d4:	f104 0347 	add.w	r3, r4, #71	; 0x47
 80012d8:	6023      	str	r3, [r4, #0]
 80012da:	6123      	str	r3, [r4, #16]
 80012dc:	2301      	movs	r3, #1
 80012de:	6163      	str	r3, [r4, #20]
 80012e0:	b002      	add	sp, #8
 80012e2:	bd70      	pop	{r4, r5, r6, pc}
 80012e4:	ab01      	add	r3, sp, #4
 80012e6:	466a      	mov	r2, sp
 80012e8:	f7ff ffca 	bl	8001280 <__swhatbuf_r>
 80012ec:	9900      	ldr	r1, [sp, #0]
 80012ee:	4605      	mov	r5, r0
 80012f0:	4630      	mov	r0, r6
 80012f2:	f7ff fa73 	bl	80007dc <_malloc_r>
 80012f6:	b948      	cbnz	r0, 800130c <__smakebuf_r+0x44>
 80012f8:	f9b4 300c 	ldrsh.w	r3, [r4, #12]
 80012fc:	059a      	lsls	r2, r3, #22
 80012fe:	d4ef      	bmi.n	80012e0 <__smakebuf_r+0x18>
 8001300:	f023 0303 	bic.w	r3, r3, #3
 8001304:	f043 0302 	orr.w	r3, r3, #2
 8001308:	81a3      	strh	r3, [r4, #12]
 800130a:	e7e3      	b.n	80012d4 <__smakebuf_r+0xc>
 800130c:	4b0d      	ldr	r3, [pc, #52]	; (8001344 <__smakebuf_r+0x7c>)
 800130e:	62b3      	str	r3, [r6, #40]	; 0x28
 8001310:	89a3      	ldrh	r3, [r4, #12]
 8001312:	6020      	str	r0, [r4, #0]
 8001314:	f043 0380 	orr.w	r3, r3, #128	; 0x80
 8001318:	81a3      	strh	r3, [r4, #12]
 800131a:	9b00      	ldr	r3, [sp, #0]
 800131c:	6163      	str	r3, [r4, #20]
 800131e:	9b01      	ldr	r3, [sp, #4]
 8001320:	6120      	str	r0, [r4, #16]
 8001322:	b15b      	cbz	r3, 800133c <__smakebuf_r+0x74>
 8001324:	f9b4 100e 	ldrsh.w	r1, [r4, #14]
 8001328:	4630      	mov	r0, r6
 800132a:	f000 f88d 	bl	8001448 <_isatty_r>
 800132e:	b128      	cbz	r0, 800133c <__smakebuf_r+0x74>
 8001330:	89a3      	ldrh	r3, [r4, #12]
 8001332:	f023 0303 	bic.w	r3, r3, #3
 8001336:	f043 0301 	orr.w	r3, r3, #1
 800133a:	81a3      	strh	r3, [r4, #12]
 800133c:	89a0      	ldrh	r0, [r4, #12]
 800133e:	4305      	orrs	r5, r0
 8001340:	81a5      	strh	r5, [r4, #12]
 8001342:	e7cd      	b.n	80012e0 <__smakebuf_r+0x18>
 8001344:	08000635 	.word	0x08000635

08001348 <__malloc_lock>:
 8001348:	4801      	ldr	r0, [pc, #4]	; (8001350 <__malloc_lock+0x8>)
 800134a:	f7ff ba45 	b.w	80007d8 <__retarget_lock_acquire_recursive>
 800134e:	bf00      	nop
 8001350:	20000090 	.word	0x20000090

08001354 <__malloc_unlock>:
 8001354:	4801      	ldr	r0, [pc, #4]	; (800135c <__malloc_unlock+0x8>)
 8001356:	f7ff ba40 	b.w	80007da <__retarget_lock_release_recursive>
 800135a:	bf00      	nop
 800135c:	20000090 	.word	0x20000090

08001360 <_free_r>:
 8001360:	b537      	push	{r0, r1, r2, r4, r5, lr}
 8001362:	2900      	cmp	r1, #0
 8001364:	d048      	beq.n	80013f8 <_free_r+0x98>
 8001366:	f851 3c04 	ldr.w	r3, [r1, #-4]
 800136a:	9001      	str	r0, [sp, #4]
 800136c:	2b00      	cmp	r3, #0
 800136e:	f1a1 0404 	sub.w	r4, r1, #4
 8001372:	bfb8      	it	lt
 8001374:	18e4      	addlt	r4, r4, r3
 8001376:	f7ff ffe7 	bl	8001348 <__malloc_lock>
 800137a:	4a20      	ldr	r2, [pc, #128]	; (80013fc <_free_r+0x9c>)
 800137c:	9801      	ldr	r0, [sp, #4]
 800137e:	6813      	ldr	r3, [r2, #0]
 8001380:	4615      	mov	r5, r2
 8001382:	b933      	cbnz	r3, 8001392 <_free_r+0x32>
 8001384:	6063      	str	r3, [r4, #4]
 8001386:	6014      	str	r4, [r2, #0]
 8001388:	b003      	add	sp, #12
 800138a:	e8bd 4030 	ldmia.w	sp!, {r4, r5, lr}
 800138e:	f7ff bfe1 	b.w	8001354 <__malloc_unlock>
 8001392:	42a3      	cmp	r3, r4
 8001394:	d90b      	bls.n	80013ae <_free_r+0x4e>
 8001396:	6821      	ldr	r1, [r4, #0]
 8001398:	1862      	adds	r2, r4, r1
 800139a:	4293      	cmp	r3, r2
 800139c:	bf04      	itt	eq
 800139e:	681a      	ldreq	r2, [r3, #0]
 80013a0:	685b      	ldreq	r3, [r3, #4]
 80013a2:	6063      	str	r3, [r4, #4]
 80013a4:	bf04      	itt	eq
 80013a6:	1852      	addeq	r2, r2, r1
 80013a8:	6022      	streq	r2, [r4, #0]
 80013aa:	602c      	str	r4, [r5, #0]
 80013ac:	e7ec      	b.n	8001388 <_free_r+0x28>
 80013ae:	461a      	mov	r2, r3
 80013b0:	685b      	ldr	r3, [r3, #4]
 80013b2:	b10b      	cbz	r3, 80013b8 <_free_r+0x58>
 80013b4:	42a3      	cmp	r3, r4
 80013b6:	d9fa      	bls.n	80013ae <_free_r+0x4e>
 80013b8:	6811      	ldr	r1, [r2, #0]
 80013ba:	1855      	adds	r5, r2, r1
 80013bc:	42a5      	cmp	r5, r4
 80013be:	d10b      	bne.n	80013d8 <_free_r+0x78>
 80013c0:	6824      	ldr	r4, [r4, #0]
 80013c2:	4421      	add	r1, r4
 80013c4:	1854      	adds	r4, r2, r1
 80013c6:	42a3      	cmp	r3, r4
 80013c8:	6011      	str	r1, [r2, #0]
 80013ca:	d1dd      	bne.n	8001388 <_free_r+0x28>
 80013cc:	681c      	ldr	r4, [r3, #0]
 80013ce:	685b      	ldr	r3, [r3, #4]
 80013d0:	6053      	str	r3, [r2, #4]
 80013d2:	4421      	add	r1, r4
 80013d4:	6011      	str	r1, [r2, #0]
 80013d6:	e7d7      	b.n	8001388 <_free_r+0x28>
 80013d8:	d902      	bls.n	80013e0 <_free_r+0x80>
 80013da:	230c      	movs	r3, #12
 80013dc:	6003      	str	r3, [r0, #0]
 80013de:	e7d3      	b.n	8001388 <_free_r+0x28>
 80013e0:	6825      	ldr	r5, [r4, #0]
 80013e2:	1961      	adds	r1, r4, r5
 80013e4:	428b      	cmp	r3, r1
 80013e6:	bf04      	itt	eq
 80013e8:	6819      	ldreq	r1, [r3, #0]
 80013ea:	685b      	ldreq	r3, [r3, #4]
 80013ec:	6063      	str	r3, [r4, #4]
 80013ee:	bf04      	itt	eq
 80013f0:	1949      	addeq	r1, r1, r5
 80013f2:	6021      	streq	r1, [r4, #0]
 80013f4:	6054      	str	r4, [r2, #4]
 80013f6:	e7c7      	b.n	8001388 <_free_r+0x28>
 80013f8:	b003      	add	sp, #12
 80013fa:	bd30      	pop	{r4, r5, pc}
 80013fc:	20000084 	.word	0x20000084

08001400 <_read_r>:
 8001400:	b538      	push	{r3, r4, r5, lr}
 8001402:	4d07      	ldr	r5, [pc, #28]	; (8001420 <_read_r+0x20>)
 8001404:	4604      	mov	r4, r0
 8001406:	4608      	mov	r0, r1
 8001408:	4611      	mov	r1, r2
 800140a:	2200      	movs	r2, #0
 800140c:	602a      	str	r2, [r5, #0]
 800140e:	461a      	mov	r2, r3
 8001410:	f7fe ff40 	bl	8000294 <_read>
 8001414:	1c43      	adds	r3, r0, #1
 8001416:	d102      	bne.n	800141e <_read_r+0x1e>
 8001418:	682b      	ldr	r3, [r5, #0]
 800141a:	b103      	cbz	r3, 800141e <_read_r+0x1e>
 800141c:	6023      	str	r3, [r4, #0]
 800141e:	bd38      	pop	{r3, r4, r5, pc}
 8001420:	20000098 	.word	0x20000098

08001424 <_fstat_r>:
 8001424:	b538      	push	{r3, r4, r5, lr}
 8001426:	4d07      	ldr	r5, [pc, #28]	; (8001444 <_fstat_r+0x20>)
 8001428:	2300      	movs	r3, #0
 800142a:	4604      	mov	r4, r0
 800142c:	4608      	mov	r0, r1
 800142e:	4611      	mov	r1, r2
 8001430:	602b      	str	r3, [r5, #0]
 8001432:	f7fe ff74 	bl	800031e <_fstat>
 8001436:	1c43      	adds	r3, r0, #1
 8001438:	d102      	bne.n	8001440 <_fstat_r+0x1c>
 800143a:	682b      	ldr	r3, [r5, #0]
 800143c:	b103      	cbz	r3, 8001440 <_fstat_r+0x1c>
 800143e:	6023      	str	r3, [r4, #0]
 8001440:	bd38      	pop	{r3, r4, r5, pc}
 8001442:	bf00      	nop
 8001444:	20000098 	.word	0x20000098

08001448 <_isatty_r>:
 8001448:	b538      	push	{r3, r4, r5, lr}
 800144a:	4d06      	ldr	r5, [pc, #24]	; (8001464 <_isatty_r+0x1c>)
 800144c:	2300      	movs	r3, #0
 800144e:	4604      	mov	r4, r0
 8001450:	4608      	mov	r0, r1
 8001452:	602b      	str	r3, [r5, #0]
 8001454:	f7fe ff73 	bl	800033e <_isatty>
 8001458:	1c43      	adds	r3, r0, #1
 800145a:	d102      	bne.n	8001462 <_isatty_r+0x1a>
 800145c:	682b      	ldr	r3, [r5, #0]
 800145e:	b103      	cbz	r3, 8001462 <_isatty_r+0x1a>
 8001460:	6023      	str	r3, [r4, #0]
 8001462:	bd38      	pop	{r3, r4, r5, pc}
 8001464:	20000098 	.word	0x20000098

08001468 <_init>:
 8001468:	b5f8      	push	{r3, r4, r5, r6, r7, lr}
 800146a:	bf00      	nop
 800146c:	bcf8      	pop	{r3, r4, r5, r6, r7}
 800146e:	bc08      	pop	{r3}
 8001470:	469e      	mov	lr, r3
 8001472:	4770      	bx	lr

08001474 <_fini>:
 8001474:	b5f8      	push	{r3, r4, r5, r6, r7, lr}
 8001476:	bf00      	nop
 8001478:	bcf8      	pop	{r3, r4, r5, r6, r7}
 800147a:	bc08      	pop	{r3}
 800147c:	469e      	mov	lr, r3
 800147e:	4770      	bx	lr
